:020000040000FA
:1000000080315828FF3FFF3F7E1480312700931D29
:1000100012282100101E122887317A2780312700EC
:10002000931156282000921C1E282100921C1E2885
:10003000A131212180312000921056282000111C6E
:100040002A282100111C2A28A031592080312000A3
:10005000111056282000131E36282100131E3628A2
:10006000BE31722680312000131256282000141E43
:1000700056282100141E5628200005304E11730208
:10008000031C4728210038082000DA004928DA013B
:100090004E15730803194E1D4F2821001412A83164
:1000A000F620EE3028009900200014127E1009007E
:1000B00088310628661DA72804307102031C6228B7
:1000C0000330F10070087106FC397106F000710808
:1000D0002200EF0047309F31032780315A30220041
:1000E000EF0046309F310327803192314122803129
:1000F000700803392400CC0051309531E32580315C
:1001000024004C0603198628FF309928700803390B
:10011000CC0051309531E325803124004C06031D7D
:100120009F2850309531E32580315A3A03199F2892
:100130005A302200EF0050309F3103278031AE311A
:100140000C268031AE31F3268031BC31632CE61DA4
:10015000FC28FF30F10704307102031CB128F101C3
:10016000F10A58087106FC397106D80003392400D9
:10017000CC0049309531E325803124004C06031929
:10018000DA2897318427803149309F310327803125
:100190009731D62780319F3103278031B6317D26B4
:1001A0008031AE31F3268031983177208031AE3105
:1001B0000C268031A831722080319531E3258031C1
:1001C00024004C060319E628FF30F828A8317220D5
:1001D00080319531E325803124004C06031DD82958
:1001E00054309531E32580315A3A0319D8295A30D1
:1001F0002200EF005430D529681C1B290430F10778
:1002000071082300A10071082200EF0053309F31D4
:1002100003278031A831A62080319F310327803108
:1002200002302500A200A3012200EF0055309F31CB
:1002300003278031A228661E372908307102083052
:10024000031CF10080307102031C28297F30F1006B
:1002500071352100EB006B082200EF0030309F3138
:10026000032780315A302200EF002F30D529E61EB7
:10027000792905307102031C3F290430F10071080F
:100280002100EC0071082200EF002E309F3103277F
:1002900080315A302200EF002D309F31032780310A
:1002A0002E309531E3258031013A031D592928303C
:1002B00073292E309531E3258031023A031D6229DE
:1002C000503073292E309531E3258031033A031DD8
:1002D0006B29803073292E309531E3258031043A23
:1002E000031D7529A0302100EC00B7314227803171
:1002F000D829661F902997307102031C81299630F6
:10030000F10071352100E80068082200EF00753027
:100310009F31032780315A302200EF007430D529F5
:10032000671FA12971082100EF006F082200EF006C
:1003300034309F31032780315A302200EF003330B0
:10034000D529E71FB22971082100DC0071082200BD
:10035000EF0036309F31032780315A302200EF0002
:100360003530D529681DC4297108E73C2100DB0020
:100370005B082200EF0016309F31032780315A308E
:100380002200EF001530D529E81CD8297108E73C78
:100390002100DA005A082200EF0018309F310327AD
:1003A00080315A302200EF0017309F31032780310F
:1003B00046276712E7126711E711A83188208031BC
:1003C000A831BC2080316811E8104B124B11CB10C2
:1003D000C81048114810491121009214842E2000A1
:1003E000D7145D082100C7007408C600892E752740
:1003F0008031CC36890BF92902304C06031D972A2F
:100400002000630C890CA831282080310730CD36BC
:10041000890B072A4D08A831582080314908A83196
:10042000B6208031C900630C682780317408CE0083
:100430000630CE36890B192A4E0801394D06CF00F9
:10044000CF0ECF0DCF0D2000490824004F06BF3935
:100450004F06A831B02080310630CC36890B2D2ACA
:100460004C080139CD00CD0CCD0C200049082400EA
:100470004D067F394D06A831B02080310430CC368E
:10048000890B3F2A01304C05CD002000600E013958
:1004900024004D06CE0020004A0824004E06FE39F6
:1004A0004E062000CA004A115F1A57185A2A013016
:1004B0004A15CA066308A831282080310530CD3698
:1004C000890B5F2A4D080139A831582080314A082C
:1004D000A831B6208031CA006F274C080339CD00FF
:1004E000CD0ECD0D20004B0824004D069F394D0642
:1004F0002000CB00A831C220803120004C0C890C98
:10050000033924004C060319882A2100D536D40C5F
:100510002000A831C2208031CC0DCC0D20004C0829
:1005200024004C06F3394C062000CC00892E752798
:100530008031CC36890B992A03304C06031D892E55
:100540002000D71CEF29A831DC208031031DEF29C2
:10055000210046087406031DEF292000D710F41B64
:10056000692C0330F436F43674052400CC00033AC9
:10057000031D3E2BA83142208031031DC32ACF30FA
:100580002000E305FF2A07307405CC004C0BCC2A71
:100590009731CD278031D52AA8317D208031031DA8
:1005A000D72A20006308CF392038E300FF2AA8317A
:1005B0006D208031031DE02A30302000E304FF2A43
:1005C000A831CD208031031DE82A20006313FF2AC3
:1005D000A8314C208031031DF02A20006317FF2A28
:1005E000A83147208031031DF82A2000E417FF2A94
:1005F000A83178208031031DFF2A200065142000D7
:10060000630E03392400CC0004309531E32580319A
:1006100024004C0603191C2B2000630E0339220012
:10062000EF0004309F31032780315A302200EF0061
:1006300003309F31032780312000630EA8319A20B8
:10064000803106309531E325803124004C060319B2
:100650003A2B00302000631B01302200EF000630EF
:100660009F31032780315A302200EF0005309F313F
:1006700003278031983177208031052CA831D22092
:100680008031031D722BA83142208031031D4B2B7A
:100690002000E714052C07307405CC004C03031D23
:1006A0005A2B20007F3067149531E32580312100DB
:1006B000C500052CA8317D208031031D622B200050
:1006C000E617052CA8316D208031031D6A2B200010
:1006D0006815052CA831CD208031031D052C200084
:1006E000E814052C03307405CC004C0BB82B0730F4
:1006F000F436F4367405CC00053A031D822B200035
:10070000E8119B2BA83147208031031D8A2B200044
:10071000E8159B2BA83178208031031D9B2B2000EE
:10072000E41522001B30EF01EF0A9F3103278031CF
:100730009D310C2580312000680C68270C309531E4
:10074000E325803124004D060319052C00302000DC
:10075000E81901302200EF000C309F31032780316F
:100760005A302200EF000B309F3103278031052CD7
:1007700074080339031D052CA83142208031031D64
:10078000CE2B2000641722001C30EF01EF0A9F31AE
:10079000032780319D310C258031052C07307405ED
:1007A000CC004C0BD62B2000E514052CA8317D2065
:1007B0008031031DDE2B20006515052CA8316D202E
:1007C0008031031DE62B2000E515052CA831CD2036
:1007D0008031031DEE2B20006516052CA8314C201E
:1007E0008031031DF62B2000E516052CA83147208B
:1007F0008031031DFE2B20006517052CA8317820C1
:100800008031031D052C2000E51721004408031D3D
:10081000602C2000660D660D01392400CC002000FC
:10082000650CA8312E208031650CA8311C20803148
:10083000650C01392400D0002000640E890C890C5D
:1008400001392400D1002000650801392400D200BC
:100850002000640D640D0139240052075107A831AE
:10086000662080312000670C01392400CC00200074
:10087000650D650D01392400CD002000650E890C41
:10088000A83182208031650EA8311C208031650E90
:1008900001392400D00020006708013924005007E6
:1008A0004F07A83151208031680C01392400CC0059
:1008B0002000680C890C013924004C072100C40772
:1008C00002304402031C842E462780316811E81050
:1008D000822EC03074052400CC00803A031D5A2DAE
:1008E000A8315F208031031D952CA8314220803132
:1008F000031D7D2C20006716172D07307405CC00D2
:100900004C0B852C2000E716172DA8317D20803157
:10091000031D8D2C20006715172DA8316D20803107
:10092000031D172D2000E715172DA831D220803187
:10093000031DBA2CA83142208031031DA22C2000B7
:10094000E616172D07307405CC004C0BAA2C20009E
:100950006616172DA8317D208031031DB22C200092
:100960006617172DA8316D208031031D172D20002B
:100970006717172D03307405CC004C0BC72CA8311A
:1009800042208031031D172D2000E717172D740812
:100990000339031D172DA83142208031031DD32CAC
:1009A00020005F12F92C07307405CC004C0BE82CAA
:1009B00020005F169F31E4278031B130EF01EF0A4C
:1009C0009F310327803122008E1420004817F92C14
:1009D000A8316D208031031DF92C200064162200FF
:1009E0003B30EF01EF0A9F31032780319D310C2509
:1009F000803120005F0E01392400CC003830953161
:100A0000E325803124004C060319172D0030200007
:100A10005F1A01302200EF0038309F310327803108
:100A20005A302200EF0037309F31032780312100F8
:100A30004408031D4D2D2000670C68272000670C1B
:100A4000A83182208031670EA8311C208031670ECA
:100A5000013924004F074E074D072100C400200034
:100A6000670EA8319A2080312000660E890C890C0F
:100A700001392400CD002000660E01392400CE008B
:100A80002000660E890C01392400A83151208031E4
:100A9000670D670D01392100C40702304402031CB1
:100AA000842E20006712E7126711E711A831BC20DD
:100AB0008031822EC0307405CC00C03A031D842ED4
:100AC000A8315F208031031DA42D61278031031DD3
:100AD0006C2D20006614892DA8314C208031031D17
:100AE000752DFC302000DE05892DA831472080318E
:100AF000031D7F2D20005E08FC390138882DA831A8
:100B000078208031031D892D20005E08FC390238D1
:100B1000DE0020005E0803392400CC003F30953110
:100B2000E325803124004C0603195D2E20005E0869
:100B300003392200EF003F309F31032780315A30C4
:100B40002200EF003E305A2EA831D2208031031D02
:100B5000EB2D61278031031DB02D2000E614CD2D33
:100B6000A8314C208031031DB92DF9302000E40557
:100B7000CD2DA83147208031031DC32D20006408EE
:100B8000F9390238CC2DA83178208031031DCD2DC4
:100B900020006408F9390438E4002000640C0339AB
:100BA0002400CC0043309531E325803124004C06ED
:100BB00003195D2E2000A831C82080319F31032702
:100BC0008031A831EE2080319F310327803196316A
:100BD0007B2680315D2E03307405CC004C0B072E34
:100BE00061278031031DF72D200066155D2EA83189
:100BF0004C208031031DFF2D2000E6155D2EA8310D
:100C000047208031031D5D2E200068145D2E74087E
:100C10000339031D5D2E61278031031D122E200034
:100C2000DE11482EA8314C208031031D1A2E2000E1
:100C3000DE15482EA83147208031031D352E2200B5
:100C400041084204031D352EE130C1000230C200CC
:100C500008302000E1060030E11901302200EF00E9
:100C60004B309F3103278031482E07307405240014
:100C7000CC00073A031D482E2000E41622004C3019
:100C8000EF01EF0A9F31032780319D310C25803120
:100C900020005E0C68274A309531E325803124001E
:100CA0004D0603195D2E00302000DE1901302200B0
:100CB000EF004A309F310327803121004408031D93
:100CC0007A2E2000680801392400CC002000660C30
:100CD000A8312E208031660CA8311C208031660C92
:100CE00001392400D0002000660801392400A83111
:100CF0006620803102304402031C842E2000A8317B
:100D0000882080312100C40121000C150E14200020
:100D1000D417AB310D23803120005F1A922EA931F8
:100D2000582180318A31912280318D31F8258031EE
:100D300020005F1EB02E5E08402780310318B02EC1
:100D4000A83122208031B3309531E3258031013A3A
:100D50000319B02EA831D72080319F31032780316D
:100D600020004F1C57190800CA1E0800A1309531F9
:100D7000E32580312400CC0020004D08A831362026
:100D80008031CD00CD1BCB2EA2309531E3258031B3
:100D90002000DC00CC2EDC01A3309531E32580312E
:100DA0002400CC0020004A08A83136208031CA0037
:100DB000A4309531E3258031A831152080314808D1
:100DC000A8318E208031C800A5309531E3258031CF
:100DD000A831152080314908A8318E208031C90002
:100DE000A6309531E3258031A8313C2080314B0875
:100DF000A831AA208031CB00A7309531E32580317E
:100E00002400CC0020004808A83136208031C800DA
:100E100062080F392400CC0005304C02031C162F49
:100E2000A8309531E325803125009200A930953115
:100E3000E3258031A8313C208031490824004C064C
:100E4000DF394C062000C900CD1C282F0130292F86
:100E500000302400CC0020004D1C302F0130312FF9
:100E6000003024004C0603190800A831A020080017
:100E7000CD302000C100CC30C2003D30C30008009E
:100E800003392400CC0002304C0208002000E41397
:100E90006510E6136710E710E5106511E51165129E
:100EA000E5126513E51308004D0801392400CC0054
:100EB0007408CD000130CD36CD364D05CE004C0640
:100EC00008000730F436F4367405CC00043A080004
:100ED0002400CC00CC0C4C0C0139CD000800740867
:100EE0002400CC00CC36CC36080020005D0824005D
:100EF000CC0006342000D018D32F8C199F2F280047
:100F00001208F500F6017608F80021004208750283
:100F1000F700031CF8037808803AF9008030790262
:100F2000031D942F41087702031C9F2F2000CD162C
:100F30009501280012082100C2002800920120001B
:100F40008C1D08000E301502031C080028009201B9
:100F500020001508D6000E305602031CB52F1F3096
:100F6000560223300318B62FBE2F23305602031C1F
:100F7000C02FBF3056020318C02F0E302100C10011
:100F80002000550CF500F50C750C0F39013A031DC6
:100F9000D02F55080739043A031DD02F2100C10175
:100FA0002100C20108008C190800EC3028009200D2
:100FB0009101200050152100D9030800C8340034E5
:100FC000163400342534003402340034043401343F
:100FD000063408340B340A34063404341E34013425
:100FE000043408343D341A340534013403340C34E9
:100FF0003E34013401341E3440343D34553402341F
:10100000FE0012001E00FE0B012800340130FA0021
:10101000DE30840087308500CE30860000308700C7
:1010200022308831002088310130840090308500E2
:1010300052308600013087001D3088310020883111
:1010400023008030EA01EB004030EC008030ED01FD
:10105000EE003F30EF004830F001F101F201F30102
:10106000F401840000308500213098310720883158
:10107000A0308400003085002E3098310720883160
:1010800020308400013085003230983107208831CB
:10109000A0308400013085003B3098310720883132
:1010A00020308400023085001F30983107208831BD
:1010B000A03084000230850040309831072088310C
:1010C000203084000330850040309831072088317B
:1010D0007E1020006B2821008E01B53172258831E9
:1010E00020004F1C7628B02188310629481C7B2817
:1010F00098310D2088312000CA1E84289831312073
:1011000088312100B401B5012921AB310D2388318B
:1011100020005F1A8E28A931582188319122883108
:10112000F82588310921883120004B1EBE28073060
:1011300073020318BD28CD1B4F1BB02835309531E5
:10114000E32588315A3A031DAA2836309531E32524
:101150008831AB2806302100DC0020004F17BE2864
:101160004F1FBE2821005C08031DBE280830200048
:10117000E8062100DC01DC0ABE284F13A431232439
:10118000883109218831292188312000CD19CC28C6
:10119000C2307302031CCF2873268831CD11210081
:1011A0009D18E02820004D1BE0287A2688312F0862
:1011B0002200B60020002E082200B50020004D17A6
:1011C0002000531CE628AA2620005310B031D92055
:1011D0008831092188312100141AF128AC31D82432
:1011E0008831292188310230210035025930031914
:1011F000340203180629A1319421883120005419A2
:101200000629FF30250096002000D41009218831DE
:1012100070282000CD1E152997319C2788319631E2
:10122000EE26883120004F101E292100320F1B2985
:10123000330A03191E29B20A0319B30A20004E1EED
:1012400008009731DA278831CA2720004F10BD31B6
:10125000462D2000491961294E14DE195329CD1C51
:101260003329013034290030A700571C39290130B7
:101270003A2900302706031DCC1E4029EE2688316E
:101280002000CD1C4529013046290030A700571CFD
:101290004B2901304C290030270603194C1E6129C7
:1012A000EE268831612921003B0B592920004C1F73
:1012B00050292000CC1E5E294C1361294C1E612947
:1012C0004C1720004E1C792973080319722900302D
:1012D00021002D02F63003192C02031C7229F5306F
:1012E000AC00AD0121002C082D04031D792920003C
:1012F000CD1320004919CD13CD1B4F1DA12922006C
:101300003F084004031DA1297235203E86000330AA
:101310008700403FBD00413FBE007235A7313A27EC
:101320008831AB0004307202031898292000CB15D5
:10133000DC302200BF000B30C00020004F11210024
:10134000CA012000CD1B08004F15CB1122003F0819
:101350004004031908000130BF020030C03B080000
:101360002100AA01AB0120004A10CA104813CA117B
:101370004A12C912491322008E1020004A1DC329A7
:1013800022000E15C52922000E118E117308031DAF
:10139000232A7208031D232A20004D1CD229200075
:1013A000CD14D4292000CD104D114B119631E826D3
:1013B000883120005315CE10CD13CD15CE1DE42954
:1013C0002100921BE42992102100921322278831D8
:1013D000031DEC2957180E2A21004E084F04031D47
:1013E0000E2A2000CD1CF9293D002008E0390D38D7
:1013F000A0002000CD18012A3D001208E0390D3868
:101400009200432288312000D41C202A22000C1193
:101410000E10E0303D00A0059205202A21004E0864
:101420004F040319182A0130CE020030CF3B202A86
:10143000222788310319571C202A22000C110E1074
:1014400078228831402AFF302100CE00CF00540896
:101450005504031D352A9631E826883197319627A1
:101460008831003068238831F30022006608670461
:10147000031D402A7308031D402AF2012000D901F0
:101480002C00980108002000D4180800210037081B
:10149000031D762A250016080319502A9603552A9B
:1014A0001608031D552A2000D41421005E08B70039
:1014B00020004F18712A17278831031D622A210046
:1014C000B736712AA73192278831031D712A21006E
:1014D00037082000A700A736A736270821003702C3
:1014E000B7002000611E0800A731EF2FB7030800E6
:1014F0002000CB18862ACE18080022000C103D00D0
:10150000900122008C103D0091010800CE180800C7
:1015100022000C143D00900122008C143D0091012A
:10152000080020005E0E0F39013A031D9F2A491E54
:10153000C91D9C2A0130C806B82688313A2B5E0E98
:101540000F39023A031DA92A491EC91D9C2A0430DD
:10155000C62A5E0E0F39033A031DB32A491EC91D60
:101560009C2A02309B2A5E0E0F39043A031DBD2AC5
:10157000491EC91D9C2A04309B2A5E0E0F39053A6C
:10158000031DC82A491EC91D9C2A0230CB069C2A6D
:101590005E0E0F39063A031DD52A491EC91DD22AEF
:1015A0002030C906B82688312E2B5E0E0F39073A37
:1015B000031DF42A491EC91DDF2A2030C906B8269A
:1015C00088315C080319EA2A22008E11AC31C82444
:1015D00088313A2B7308031D3A2B2100300831045F
:1015E000031D3A2B20002E2B5E0E0F39083A031DE7
:1015F0000F2B491EC91DFE2A2030C906B826883186
:101600005C080319082BC91EE42A22008E15E62A5D
:101610007308031D3A2B210030083104362B5E0E6F
:101620000F39093A031D1F2B491EC91D192B2030E4
:10163000C906B8268831CD1C5419332B2E2B5E0ECB
:101640000F390A3A031D3A2B491EC91D292B203098
:10165000C906B8268831CD185419332BC91E382B2A
:1016600022008E153A2B5E080339023A031D3A2BED
:1016700022008E112000490E890C01392300E80058
:10168000A9309531E3258831230068060319522BD0
:1016900000302000C91A01302200EF00A9309F312C
:1016A000032788312000480801392300E800A730CB
:1016B0009531E325883123006806031908000030BE
:1016C0002000481801302200EF00A7309F31032F7F
:1016D0002000C700E026883120004C08240048067E
:1016E000FC3948062000CC004D1E812B0330210020
:1016F000A800A90120004708031D6F2D4527883148
:101700006F2DCD1BDF2C2300230822006F0203184E
:10171000A02B6F08200047020318A02B4B0E890C4A
:1017200003390319A02B172788310319A02B4B0E5F
:101730002400C800480C0339C800C803F9268831C2
:101740004F2788310318A72B21005B08AE2B4708D1
:1017500022006F020318B02B21005A08A800A9012B
:101760002000E0268831023048020318ED2B4F2775
:1017700088310318ED2B2C278831031DC42B210041
:101780005B08A8000230D52B31278831031DCD2BF3
:1017900021005B08A8000430D52B27278831031DC2
:1017A000DA2B21005B08A8000630A901A80703185E
:1017B000A90A432C042788314908803ACA0080309E
:1017C0004A02031DE72B22006F0824004802031C75
:1017D000432C02302100A800422C2000E026883152
:1017E000023048020318432C4A2788310318432C3F
:1017F0002300280822006F020318082C6F0823001A
:1018000025020318082C0C302100A800A9013B2C4C
:101810003B278831031D112C21005A08A8000230F3
:10182000192C40278831031D1B2C21005A08A800C1
:101830000330A901382C2C278831031D252CC926FB
:101840008831031CA9030430382C31278831031D4B
:101850002F2CC9268831031CA9030530382C2727D3
:101860008831031D3B2CC9268831031CA90306308F
:10187000A8070318A90A362788310318432C21002A
:10188000A801A80AA90136278831031CAF2CA7316B
:1018900059278831031D652C22006F08230026027A
:1018A0000318652C210029082400C90021002808FC
:1018B0002400C800C936C80C480821002802A80026
:1018C000240049082100293BA9002000A7319227C4
:1018D0008831031D7B2C2300290822006F02031886
:1018E000732C0630742C03302000A700D626AE31AE
:1018F000DE268831E6262000A831E5208831031D48
:10190000982C23002A0822006F020318912C0C3017
:101910002000A700D626AE31DE268831E6268831A3
:10192000982C2100A835A90DA835A90DA835A90D19
:1019300020004B0E890C0339031DAF2C23002B080C
:1019400022006F020318A62C1330A72C0E302000A3
:10195000A700D626AE31DE268831E6268831210062
:1019600029082000B000210028082000AF00E7254A
:101970009F31C427883123006D082000C100230057
:101980006E082000C20023006F082000C3009531BC
:10199000F52588319F31592788319C31A824883119
:1019A00065082100A900230064082100A800200088
:1019B0004C0803392400C800F92688315E2D220026
:1019C0003E082100A90022003D082100A8000030A7
:1019D00022003E02023003193D02031C592D200053
:1019E000CB19592D272788310319042D102D2100DB
:1019F0005008A8075108582D0E278831362D210090
:101A00005208A8075308582D70080339013A0319E2
:101A1000F72C033A0319FC2C013A0319FF2C592D1A
:101A200031278831031D1A2D68082100A8072200DC
:101A30006908572D2C2788310319FF2C402788313E
:101A40000319FF2C3B2788310319F72C23002608A4
:101A500022006F060319FC2C2300270822006F06C2
:101A6000031D3E2D0E278831C936C80CC936C80C57
:101A700048082100A80724004908572D23002808FA
:101A800022006F06031D592D06302000A700A80173
:101A9000210051082000AA00210050082000A900C0
:101AA000C225883127082100A80720002808210026
:101AB000A93D20004D1D5E2D4527883136278831F0
:101AC00003186F2D2000CE1F6F2D2100A801A90142
:101AD00020005C08031D6F2D2200EF01EF0AA731E3
:101AE000F827883103193506031D802DEF303302A6
:101AF000FF3003193202031C802DA801A80AA90196
:101B00004A27883103188A2D2000CD1F4D198A2DB0
:101B10002200EF0A22006F08200047020318922DCE
:101B20002200EF0320005908031DBA2D2C001808CD
:101B300022006F020318BA2D720BBA2D04278831C8
:101B400022006F08240048064904031DBA2D200016
:101B5000CF1ABA2D5A0E0F3922006F0720005B07EB
:101B60002200EF002000CF16DA01DB012100B801CE
:101B70002200D10121002908D5002808D400220024
:101B80006F080800AB01AC01270828040319E22DF7
:101B9000AD01AD0AA81BCF2DA735A80DC92DAB35BA
:101BA000AC0D28082A02031DD72D27082902031C83
:101BB000DE2D2708A9022808AA3B2B14A836A70C5B
:101BC000AD0BCF2D2C08A8002B08A70008002F086C
:101BD000A7003008A8008E30A901AA00AB019631F9
:101BE000AA262708AF002808B0002908B10008007D
:101BF00020005F080F39013A031D082E1C27883189
:101C0000A70DA70D49082706FB392706C900492E4D
:101C10005F080F39023A031D142E1C278831A70DC7
:101C20004B082706FD391F2E5F080F39033A031DA5
:101C3000222E1C278831A70E4B082706EF392706CE
:101C4000CB00492E5F080F39043A031D2F2E491F80
:101C50002C2E2000C814492E2000C810492E5F08E1
:101C60000F39053A031D3C2E491F392E2000481517
:101C7000492E20004811492E5F080F39063A031DEE
:101C8000492ECE19491F472E21009210492E2100BE
:101C900092142000D41B08005F080F39043A03197E
:101CA000562E5E0E0F39033A031D5B2EC81C5B2EA9
:101CB00021000E145D2E21000E1020005F080F3948
:101CC000053A0319682E5E0E0F39043A031D702E73
:101CD000481D6D2E21000C15080021000C11080074
:101CE00021000C1108009631E82620004D175410F1
:101CF000D3130800B001B1012200CD0A5427883166
:101D000022004D086E06031DA42E2000531422004D
:101D1000B501B6014C082000A700A80122003A082E
:101D20002000AA00220039082000A900C2252808A6
:101D3000B1002708B00031082200B80020003008A8
:101D40002200B7009631E82620003108AF003008A5
:101D5000AE000800220036082000C300220035082B
:101D60002000C200B0317E2088310921AD31222D02
:101D7000490C2300E800E80C680C0139E900E90E81
:101D80002000490823006906EF3969062000C900D0
:101D9000080021005A08A800A90120004B0E890C58
:101DA00003392400C8002100A8020800A80121006E
:101DB00029082000AA00210028082000A900080006
:101DC0004B0E890C03392400C800080028082100A4
:101DD000A900200027082100A8000800CD17DC0179
:101DE0007208D9004E304E102100AC000230AD0018
:101DF0000800C80EC80D20004B08240048069F3973
:101E000048062000CB00080023002108FF3E2400E4
:101E1000C800FF3003180030C90008002100510835
:101E20002400C900210050082400C80008004B0EFF
:101E3000890C0339033A0800490E890C890C0139D1
:101E4000A700080020005E080339023A08002300BA
:101E5000210822006F0608002300230822006F06D5
:101E600008002300220822006F0608002300210832
:101E700022006F0208002300250822006F060800D8
:101E80002300240822006F06080002302100A80069
:101E9000A90108002000470822006F020800220064
:101EA0006F0820004702080021001C082200DF0004
:101EB000DE0121001B082200DE070318DF0A2000D4
:101EC0004D175319682F23002136730203186E2F04
:101ED000200053112200B901BA01CC0122005F0891
:101EE000B8005E08B7005E08B9075F08BA3DCC0AC3
:101EF00020004D1A0800220037083804031D832FE4
:101F00002000CE17852F2000CE1352082200380261
:101F1000031D8E2F20005108220037020318A42F22
:101F2000230021087302031CA12F20005208210066
:101F30002B02031D9D2FC5278831031CA12F2000D4
:101F4000D31720005410B12F380820005202031D6F
:101F5000AD2F22003708200051020318B12FD313F0
:101F600054142300210873020318B92F2000CD1B3D
:101F7000C22F2300210873020318080020005C0808
:101F8000031D0800D3135414080020005108210039
:101F90002A02080021004308031DD92F2C082D0414
:101FA000031DD42F2000CD13200057108C1A571476
:101FB000ED2F2000571CDE2F0130DF2F0030A7004F
:101FC0008C1EE42F0130E52F003027060319ED2F7A
:101FD000210043080319ED2FC3032000571CF22FE3
:101FE0000130F32F0030A7008C1EF82F0130F92F9D
:101FF00000302706031D080038302100C300080008
:10200000FF3F003480343F346634A6343F3401341B
:10201000003402340034FF345F34013400340A34B5
:10202000003418340034CD340434023400347034B5
:1020300000340C3400347B34003401342100921815
:1020400023287027903111182A28200099019A011D
:1020500021001114FF302200EF0052309F3103277E
:102060009031C4279F310327903121000C110E10AD
:1020700022000C110E102000571C46285E08033960
:10208000023A031D462822000C150E1420004D169E
:10209000D415AE31F32690312000CE1048136208DB
:1020A0000F39013A03195D286208F0390138E2005E
:1020B0003F30E205CF30E20563106012E3112000EB
:1020C000D41D3D294B0E890C0339013E2100DD0052
:1020D0004130E325903121005D06031984287B26D9
:1020E00021005D082200EF0041309F31032790312D
:1020F0004030E32590315A3A03198428A831E12071
:1021000090319F310327903120004A1C8B286408AE
:10211000F93902389028491F92286408F93904389F
:10212000E4009428F930E405640C03392400D3005A
:102130004330E3259031240053060319B2287B264F
:10214000A831C82090319F31032790314230E325D8
:1021500090315A3A0319B228A831EE2090319F31BC
:10216000032790312000CD1EBA289C279031EE26FF
:102170009031C3282100320FC028330A0319C32825
:10218000B20A0319B30A20004E1ACE1ACB28DA2756
:10219000BD3146259031A43123249031AC31D8246F
:1021A00090312000CA1DFB285230E32590315A3A65
:1021B0000319FB28A831A62090319F3103279031C5
:1021C0007208A731432790312200EF0053309F312E
:1021D000032790312000571CF4285E080339023A87
:1021E000031DF42822000C118F312227903103198E
:1021F000FB2822000C155230E32590315A3A031D7A
:1022000020297308031D20295330E325C03C2100F9
:10221000D8001F302000A70021005808AF31A527A3
:1022200090312100D800D80A58082200EF007630FB
:102230009F3103279031B6317D2690312000D41193
:102240004B30E3259031003A031D5F2820005A30BF
:10225000D4114D122200EF0052309F3103279031EC
:102260005A302200EF0054309F31032790318427E9
:1022700074309F31032790315F284D10A631B52669
:1022800090314D12AE31F3269031F301210010123E
:102290004B30E32590312400D300D30E20004D08AD
:1022A00024005306EF3953062000CD0023003E08DA
:1022B0002100C900D401D50122003C30E601E7012C
:1022C000EE002100921866297027903120004D1EE3
:1022D000362A2200C901CA01B731F62790314908D0
:1022E00073060319802954085504031D8029E82624
:1022F00090319627210049088B3168239031F300F3
:10230000AC31D8249031210049087306031DAA2955
:1023100073080319AA291E30FA007A080319AA299A
:102320007A08A731432790317306031DA8297A083C
:102330009F3E86000108A031192090312400D3006F
:10234000D401AF31BE2790315308C03F5408C13F7C
:10235000FA038D297308031D662920005A304B119A
:10236000CE104D122200EF0050309F3103279031E4
:10237000700803392200EF0051309F31032790315C
:10238000842773309F310327903125004008410492
:10239000031DCC29FF30CD295A302200EF005430E4
:1023A0009F31032790315430E32590315A3A031D71
:1023B0002F2AFA011E30FA0A7A0203181B2A7A35EC
:1023C000A23E860002308700403F2400D300413FF8
:1023D000D4007A35A03E8600403FD500413FD6006C
:1023E00054085602031DF62953085502031CDA2926
:1023F000AF31BE279031403FD300413FD400003081
:102400005402FF30031953020318DA297A35A03E2B
:102410008600403FD300413FD4005308013ED50021
:102420000030543DD6007A35A23E86005508C03FA4
:102430005608C13FDA29FA01FA0A1F307A02031856
:102440002F2AAF31BE27903101082200EF007A0811
:10245000543E9F310327903195181D2A1C2A2200D3
:102460004B30EF019F3103279031662922000C1574
:102470000E10CF30EE01EE0A20009B052100101651
:1024800008000130E32590315A3A031D6D2A0230CD
:10249000E3259031003A0319622A0230E325903196
:1024A0002300E8006A3068020318622A0230E3253C
:1024B00090313F3A0319622A0230E32590313E3AC7
:1024C000031D6D2A3D302200EF0002309F310327AB
:1024D0009031D2279F31032790310130E32590318D
:1024E0005A3A031D772A0230E3259031782A3D308D
:1024F0002100ED005330E32590312300E800053042
:102500006802031C8C2A5330E32590312300E80035
:1025100081306802031C982AAF31FC2790319F312B
:1025200003279031A831A62090319F3103279031A5
:102530007008FC390138F000FC302000D805A030CC
:10254000E32590315A3A031DA72A2000CA164630C7
:10255000E32590315A3A031DB62A4730E3259031DE
:102560002300E8007006FC396806B92A7008FC39B7
:102570000138F0004830E32590315A3A031DC62A4D
:102580004930E325903153279031C92AFC3020008F
:10259000D8054830E32590315A3A0319E72A7330B9
:1025A000E32590312300E800043068020318E72A8D
:1025B0007330E3259031532703392200EF0049306F
:1025C0009F3103279031D6279F3103279031033065
:1025D000E32590315A3A031DF82A0430E32590315F
:1025E0002300E800E80E20006308A7279031FA2AAC
:1025F000CD279031E3000530E32590315A3A031D91
:102600000E2B0630E32590312300E800E80E692701
:102610009031BF3968062000E300102B20006313BF
:102620000730E32590315A3A031D1E2B0830E3256D
:1026300090316B2690315E2790311F2BA227D70057
:102640008731382790319F3140279031F5259F31D0
:102650004D2790310930E32590315A3A031D362B2E
:102660000A30E3259F31A4279031382BC8279031B9
:102670000B30E32590315A3A031D482B0C30E325EB
:1026800090317727903168088A279031E8004A2BEB
:102690002000E8110D30E32590315A3A031D582BE4
:1026A0000E30E32590316B269031482790315D2B19
:1026B00023002030ED01EE004130EF008731382754
:1026C00090310B279031F525903130279031113022
:1026D000E32590315A3A031D7D2B1230E3259031CA
:1026E0006B2690312F082100A00020003008210027
:1026F000A100200031082100932B70080339013A12
:10270000031D882B00302100A000A1004030932B36
:1027100070080339023A031D952B00302100A000F8
:102720004030A1004130A200992B2100A001A1015D
:10273000A2011330E32590315A3A031DAF2B143018
:10274000E32590316B2690312F082100A300200053
:1027500030082100A400200031082100C42B70089B
:102760000339013A031DBA2B21008030A301A400D4
:102770003F30C42B70080339023A031DC62B2100D9
:102780003030A301A4004130A500CA2B2100A301D1
:10279000A401A501873138279031F1269031F52524
:1027A00090311827873138279031FE269031F52552
:1027B0009031242790311530E32590315A3A031D8A
:1027C000E52B1630E3259031E62B0A302100DB00A3
:1027D0001730E32590315A3A031DF22B1830E325C8
:1027E0009031F32B0B302100DA0020005808B3277A
:1027F0009031031CFE2BFC302000D8057008B32755
:102800009031031C072C7008FC390138F000BA31F4
:102810001C2290312D30E32590315A3A031D1E2C95
:102820002E30E3259031013A031D182C28302F2C2F
:102830002E30E3259031023A031D202C50302F2CEE
:102840002E30E3259031033A031D282C80302F2CA5
:102850002E30E3259031043A031D312CA0302100A5
:10286000EC002F30E32590315A3A031D3B2C3030D9
:10287000E32590313C2C1E302100EB003130E32564
:1028800090315A3A031D482C3230E3259031492CBF
:1028900040302100E800A03CE9003330E3259031CE
:1028A0005A3A031D572C3430E3259031582C02300E
:1028B0002100EF003530E32590315A3A031D642C96
:1028C0003630E3259031652C06302100DC003730AE
:1028D000E32590315A3A031D792C3830E3259031A5
:1028E0002300E800E80E20005F08BE279031DF00DB
:1028F0007B2C20005F125F1E802C481722008E1454
:102900003C30E32590315A3A031D8B2C3D30E325B2
:10291000903109078C2C1E302100DE000A305E0247
:102920000318952C20006116972C200061123E3070
:10293000E32590315A3A031DA82C3F30E32590310E
:102940002300E80020005E087E279031DE00AB2CDB
:10295000FC302000DE054A30E32590312300E800FA
:10296000023068020318BE2C4A30E32590317727E5
:1029700090315E088A279031DE00C02C2000DE11E5
:10298000B030E32590315A3A031DD02CB130E32505
:1029900090312300E8002000600890279031D42C6B
:1029A00020006008F0390138E000B230E3259031B2
:1029B0005A3A031DEA2CB330E32590312300E80096
:1029C000E80EE80D20006008230068069F396806BD
:1029D0002000EE2C200060089F392038E000B43041
:1029E000E32590315A3A031D052DB530E32590318A
:1029F0002300E800E80DE80D2000610823006806C8
:102A0000FB3968062000E100072D20006111B63077
:102A1000E32590315A3A031D172DB730E325903145
:102A20002300E800200061087E2790311B2D200044
:102A30006108FC390138E100B830E32590315A3A99
:102A4000031D2E2DB930E32590312300E800E80E58
:102A500020006008BE279031E000302D2000601279
:102A6000C030E32590315A3A031D402DC130E32593
:102A700090312300E8002000620890279031442D17
:102A800020006208F0390138E200C230E3259031BD
:102A90005A3A031D562DC330E32590312300E80038
:102AA000E80E20006208A72790315A2D2000620806
:102AB000CF391038E200C430E32590315A3A031D73
:102AC000712DC530E32590312300E800E80EE80DB4
:102AD000E80D20006208230068063F3968062000E0
:102AE000752D200062083F394038E200C630E325EA
:102AF00090315A3A031D8A2DC730E32590312300C7
:102B0000E8002000630823006806FE3968062000FC
:102B1000E3008C2D20006310D230E32590315A3A27
:102B2000031D9E2DD330E32590312300E800692753
:102B30009031FB3968062000E300A02D20006311CE
:102B4000D430E32590315A3A031DB42DD530E32516
:102B500090312300E800E80E20005E08230068069C
:102B60000F3968062000B82D20005E080F39103894
:102B7000DE00D630E32590315A3A031DC92DD730F7
:102B8000E32590312300E80020005F089027903172
:102B9000CD2D20005F08F0390138DF00D830E32563
:102BA00090315A3A031DE02DD930E32590312300AE
:102BB000E800E80D6927F73968062000E3000800FF
:102BC0002000E31108002000A700E72D200064008A
:102BD00031009518E62D15172000270831009100C7
:102BE0007030920015141308080041082300DB0020
:102BF000200042082300DC0020004308AD2790316C
:102C0000DE005E08031D052EB92F200044082300B6
:102C1000DB00200045082300DC0020004608AD272B
:102C20009031E3006308031D162EB92F63087B3E25
:102C3000DE07200043082300E300200046082300AD
:102C4000E3068030E3052000FF30C217C517C40536
:102C5000C505C60123000730DF01E001E101E20004
:102C60002000411C352E3C2790312000C336C20C79
:102C7000C10CC435C50DC60D2300E20B302E093042
:102C8000E2002000411C462E3C2790312000C33634
:102C9000C20CC10C2300E136E00CDF0CE20B412E2C
:102CA0005F082000A700230060082000A800230080
:102CB00061082000A90023005E082000AA0023006C
:102CC00063082000AB00AA262708C1002808C2001C
:102CD0002908C30008002000B300A7008E30A80117
:102CE000A901AA00AB01AA262708AF002808B00056
:102CF0002908B1000800200091101F15FC309F0525
:102D0000640C0339013A031D8A2E1F08FC3901386F
:102D10009F00912E640C0339023A031D912E03305B
:102D20009F0487309F05C0309E00033021005D0660
:102D3000031D9C2EA030A52E02305D06031DA22E81
:102D40008030A52E5D0BA72E603020009E00200055
:102D50009D0108002A080319B22E29082804270417
:102D6000031DBA2EA701A801A9010800AA0AA936C5
:102D7000A80CA70CFE3029050319C82EB62EAA0AE6
:102D8000A70A0319A80A0319A90AA936A80CA70CAF
:102D9000FF3029050319D52EBF2E02302A02031C4D
:102DA000D72EAA03A735A80DA90DA81FCD2E2A1C22
:102DB000A813AA362A08AE00AD01AC012C08A7045E
:102DC0002D08A8042E08A9042B08031DA917080024
:102DD0002200B901BA01CD01CC010800DF27BE31C4
:102DE000A52E210020082000C40021002108200079
:102DF000C500210022082000C60008002100230889
:102E00002000C400210024082000C500210025085E
:102E10002000C600080023006D082000C400230025
:102E20006E082000C50023006F082000C6000800BF
:102E300041082100A000200042082100A10020003C
:102E400043082100A200080041082100A30020003F
:102E500042082100A400200043082100A50008002A
:102E600041082300ED00200042082300EE0020006E
:102E700043082300EF00080044082300DF07200078
:102E800045082300E03D200046082300E13D0800FE
:102E90002F082300ED00200030082300EE00200062
:102EA0003108230008002300E80020005808230010
:102EB0006806FC3968062000D80008002F082200A8
:102EC000D500200030082200D60020003108220062
:102ED0000800E80DE80D20006308230068060800DC
:102EE00028009501FF30960021009214080023006D
:102EF000E800E80DE80DE80D200008002300680652
:102F0000FC39680620000800200058080339220018
:102F1000EF00080023006806F73968062000080063
:102F200023006806F03968062000080020005315C9
:102F300073082200EF0008002100B201B301200055
:102F4000CD12080022005030D501D60041342300B4
:102F50006806CF396806200008002300DD00031052
:102F60005C0D5D0D080003392300E80004306802A1
:102F700008002000C101C201C30108002300680647
:102F8000EF39680620000800FF302200EF005434BB
:102F900070302200E800E901080020006308CF3902
:102FA000103808005A302200EF0001345A30220055
:102FB000EF0048344E122200C901CA010800243033
:102FC0005602031CEA2F413056020318EA2F210053
:102FD000401408000F305602031CF52F1E30560215
:102FE0000318F52F2100401008006F305602031C13
:102FF0000800BE305602031808002100C014080063
:10300000FF3FFF3FFF3FFF3FFF3FFF3FFF3F6400AA
:1030100080010131890B08280034541908005E082A
:103020000339023A03191A285E0E0F39013A031DBB
:1030300008002B285E0E0F39013A031D0800571CAB
:10304000282822000C1925280C150E1C0E14080027
:10305000571808002B2822000C190C110E180E10FE
:103060000800A0309531E32598315A3A0319080039
:1030700021005A30CC012200EF00A0300327983104
:10308000003020004D1801302200EF00A13003274E
:103090009831210048082200EF00A23003277F303A
:1030A0009531E32598312100480603195D28480829
:1030B0002200EF007F3003279831003020004A18AB
:1030C00001302200EF00A3300327983100302000A8
:1030D000491B01302200EF00A53003279831200062
:1030E0004B0E890C03392200EF00A630032FBE27B8
:1030F000983124279831DF2398312F082200B2001D
:10310000200030082200B300200031082200B40063
:10311000B227983124279831DF2398312F082200D5
:10312000AF00200030082200B0002000310822004B
:10313000B100AC27983124279831DF2398312F082C
:103140002200AC00200030082200AD002000310831
:103150002200AE00B827983124279831DF23983118
:103160002F082200A900200030082200AA00200019
:1031700031082200AB00BE27983132279831DF2377
:1031800098312F082300D800200030082300D900F0
:10319000200031082300DA00B22798313227983115
:1031A000DF2398312F082300D500200030082300AA
:1031B000D600200031082300D700AC2798313227F1
:1031C0009831DF2398312F082300D20020003008E7
:1031D0002300D300200031082300D400B827983101
:1031E00032279831DF2398312F082300CF002000A9
:1031F00030082300D000200031082300D1008030A7
:10320000CC01CD003F30CE000830C900CF30CA001D
:103210004730CB0033302200A600F330A700403007
:10322000A800FA011F30FA0A7A020318322B652728
:1032300096316B269831CB2798318D2498313B08F5
:10324000C1003C08C2003D08C300652796316B26CB
:103250009831CB2798318D243B08C4003C08C50029
:103260003D08C6009531F525983141082300C60078
:10327000200042082300C700200043082300C800A4
:10328000220026082000B400220027082000B500F4
:10329000220028082000B6007A08A7314327983179
:1032A00096316B2698312F08B7003008B8003108E6
:1032B000B900B23198229831031C64292300803070
:1032C000C601C7003F30C800230046082000B300F5
:1032D000230047082000B400230048082000B50060
:1032E000230049082000B60023004A082000B70048
:1032F00023004B082000B800B2311F229831330858
:103300002300C300200034082300C4002000350837
:103310002300C5004C082000BB0023004D082000FE
:10332000BC0023004E082000BD00230043082000FD
:10333000BE00230044082000BF00230045082000F1
:10334000C0008D2498313B082300C30020003C08B6
:103350002300C40020003D082300C5002000630EA8
:103360000339033A031DEF2921003A087A02031CAE
:10337000BE293D302000C1008A303D2A3A087A0239
:1033800039080318D2297A02031CD12923005808CE
:103390002000C100230059082000C20023005A0861
:1033A000A62A39087A020318E42907307A02031C96
:1033B000E429220032082000C10022003308200046
:1033C000C20022003408A62A220032082000B200DF
:1033D000220033082000B30022003408B22A630E12
:1033E0000339023A031D2F2A21003A087A02031CEE
:1033F000FE2914302000C1006E303D2A3A087A02BE
:1034000039080318122A7A02031C112A23005508CE
:103410002000C100230056082000C20023005708E6
:10342000A62A39087A020318242A07307A02031CD4
:10343000242A22002F082000C1002200300820008A
:10344000C20022003108A62A22002F082000B20064
:10345000220030082000B30022003108B22A630E97
:103460000339013A031D712A21003A087A02031C2C
:10347000402AAE302000C1000730C2003F30C12AD0
:103480003A087A0239080318542A7A02031C532A8C
:10349000230052082000C100230053082000C2006E
:1034A00023005408A62A39087A020318662A07302E
:1034B0007A02031C662A22002C082000C100220088
:1034C0002D082000C20022002E08A62A22002C0867
:1034D0002000B20022002D082000B30022002E0898
:1034E000B22A630E0339031DC72A21003A087A0263
:1034F000031C812A85302000C1006B30C2003E30A1
:10350000C12A3A087A0239080318952A7A02031C5C
:10351000942A23004F082000C100230050082000F7
:10352000C20023005108A62A39087A020318A82AE3
:1035300007307A02031CA82A220029082000C100B3
:1035400022002A082000C20022002B082000C12AE5
:10355000220029082000B20022002A082000B3001F
:1035600022002B082000B400CD30AF004C30B0005A
:103570003E30B100DF2398312F08C1003008C2006F
:10358000310878279531F525983198279831200012
:10359000631FDB2A220055082000C10022005608C4
:1035A0002000C20022005708200078279531F52519
:1035B000983198279831F6279831031DFA2A9227D7
:1035C000403FAF00413FB0008D31E7259831C4271F
:1035D0003330C100B330C2003F30C3009531F52510
:1035E000983159279831A824983192276408C03F10
:1035F0006508C13F80309531E32598315A3A031967
:10360000072B2200EF017A08803E03279831230020
:103610004308E4004408E5004508E600A824983182
:1036200092276408C03F6508C13F80309531E3258B
:1036300098315A3A031D122992279831D8277A08CF
:10364000803E9531E325983124004807CA00490897
:103650000318490ACB00922798314A08C03F4B080B
:10366000C13F1229F62798310319662B630E0339DF
:10367000031D502B26008030DA01DA0ADB01953178
:10368000E32598315A3A031D502B9D309531E3259F
:10369000983126005A07DA005B0803185B0ADB0042
:1036A00026008030DC01DC0ADD019531E32598310C
:1036B0005A3A031D662B9E309531E325983126003A
:1036C0005C07DC005D0803185D0ADD002600803021
:1036D000DE01DE0ADF019531E32598315A3A9F3049
:1036E000031D7D2B9531E325983126005E07DE0012
:1036F0005F0803185F0ADF00882B9531E3259831B6
:10370000003A0319882B22009F30EF0103279831DC
:10371000FA010730FA0A7A020318A12B922798318E
:10372000D827983103304902E93003194802031CB5
:10373000892B7A35203E8600E830C03F0330C13FF8
:10374000892B0F302600A2002830A301A4000930E5
:10375000A5019531E32598315A3A031DB62B0A305D
:103760009531E3259831A4279831B92B9731C82793
:10377000983103302000A700A801220068352000FE
:10378000A9002200690D2000AA008D31C225280859
:103790002100D300200027082100D2005308240074
:1037A000C900210052082400C800C936C80C4808C6
:1037B0002100D000240049082100D10008002F0872
:1037C000B5003008B6003108B7000310360D370DCC
:1037D000BA003208B5003308B6003408B700031049
:1037E000360D370DB9003A080319022C39083A0290
:1037F000390803180A2CB5003A08B5021930350209
:10380000031C092C3208AF003308B0003408B100A3
:1038100008003908031908003A0839020318182C5F
:103820003A08B5003908B502193035020318080006
:103830000630B800B11BB817B41B3817B017B10168
:10384000B317B40139083A0203183D2CB235B30D51
:10385000B40DB90339083A060319382CB8033808EF
:1038600007390319382C262CB136B00CAF0CBA0A24
:103870003A0839060319572C342C3A083902031830
:10388000572CAF35B00DB10DBA0339083A060319FC
:10389000532CB803380807390319532C412CB4367C
:1038A000B30CB20CB90A3A083906031D4F2CB81FE5
:1038B000622CFF30AF06B006B106AF0A0319B00A9A
:1038C0000319B10A381F6A2CDE2798310319B30A8D
:1038D0000319B40AB8012F08B2073008B33D310804
:1038E000B43DB41F7A2CDE270319B30A0319B40AB6
:1038F000B801B80A3208A7003308A8003408A900A4
:103900003A08AA003808AB009631AA262708AF006B
:103910002808B0002908B10008003D083C043B0419
:103920000319942C8030BD063E08AF003F08B0005C
:103930004008B1003B08B2003C08B3003D08B400A9
:10394000DF232F08BB003008BC003108BD00080091
:10395000862798310310400D410DC7004708031D0D
:10396000B72C2300E401E501E601E701080023008C
:10397000862798311730C136C00CBF0C890BBB2C81
:103980003F08C2002300E517E60164082400C300D5
:10399000230065082400C400230066082400C50035
:1039A0008E30C601C702C71FE12C4708803A8F3E00
:1039B000031CB12CC636C50CC40CC30CC70FDA2CC3
:1039C000EE2C183047020318B12C47080319EE2CCF
:1039D000C335C40DC50DC60DC703E52C4208031938
:1039E000FC2CC309C409C509C609C30A0319C40AC2
:1039F0000319C50A0319C60A46082300E700240074
:103A000045082300E600240044082300E5002400C4
:103A100043082300E40008001B309531E32598316A
:103A2000013A031DA72D22000430EF01EF0A0327FE
:103A3000983120006308CF391038E30022000630A7
:103A4000EF010327983120000D3063132200EF00AF
:103A5000083003279731A2279831D70087313827BC
:103A6000983140279531F52598314D2798311C30F4
:103A7000EF000A300327983170302200E8000C3044
:103A8000E901EF010327983120000A30E8112200F4
:103A9000EF000E300327983100302300ED00803016
:103AA000EE003F30EF00FF302200EF00113003271F
:103AB0009831FF302200EF0013300327983170084F
:103AC0000339013A031D712DCD302100A0004C3087
:103AD000A1003E30A200CD30A300CC30A4003D3088
:103AE000822D70080339023A031D842D9A3021007B
:103AF000A0009930A1003F30A200CD30A3008C304F
:103B0000A4003F30A5008B2D2100A001A101A2013E
:103B1000A301A401A5010A302200EF0016300327FB
:103B200098310B302200EF00183003279831FF3016
:103B30002200EF0080300327AE310C269831772029
:103B400098312000E41122001B30EF0103271C30C4
:103B50009531E3259831013A031DE02DFF30220015
:103B6000EF001D3003279831FF302200EF001F3097
:103B700003279831FF302200EF00213003279831CE
:103B8000FF302200EF00233003279831FF3022005E
:103B9000EF00253003279831FF302200EF00273057
:103BA00003279831FF302200EF0029300327BA3174
:103BB0001C2298312000641322001C30EF010327DF
:103BC0003B309531E3259831013A031D8C2E0230AC
:103BD0002200EF002E300327983150302100EC00F6
:103BE00032302200EF002F3003279831323021008D
:103BF000EB003E302200EF003230032798313E3098
:103C00002100E800A03CE90022003430EF01EF0A77
:103C10000327983121000630EF01EF0A2200EF0060
:103C200036300327983106302100DC00220038307E
:103C3000EF010327983120005F122200B130EF011D
:103C4000EF0A032798312000E4279831B330EF01C1
:103C5000EF0A0327A831222098312200B530EF0166
:103C60000327983120006111FB27983103279831F1
:103C7000F02798312200B930EF0103279831200056
:103C800060122200C130EF01EF0A032798312000B3
:103C90006208F0390138E2002200C330EF01EF0A78
:103CA00003279831EA2798312200C530EF01EF0A47
:103CB00003279831D22798312200C730EF0103271C
:103CC0009831200063102200D330EF010327983190
:103CD000200063112200D530EF01EF0A032798314D
:103CE00020005E080F391038DE002200D730EF01C7
:103CF000EF0A0327983120005F08F0390138DF0010
:103D00002200D930EF01032798312000E31164121B
:103D100022003B30EF0103274C309531E3259831E9
:103D2000013A031D08000F302200EF003D30032749
:103D300098311E302100DE0022003F30EF010327C2
:103D40009831FC302000DE0504302200EF004130C5
:103D50000327983104302100DD0022004230EF01BA
:103D60000327F9302000E40596317B269831AF31E6
:103D7000FC2798310327983122004730EF01EF0AE2
:103D8000032798317008FC390138F00022004930CF
:103D9000EF010327FC302000D805BA311C229831EE
:103DA000B6317D269831AE31F32698317720AE3189
:103DB0000C26983122004B30EF0103279831200068
:103DC000FF30E1112200EF00503003279831FF301F
:103DD0002200EF00513003279731C4279831032781
:103DE0009831FF302200EF00733003279831FF3005
:103DF0002200EF007630032798312000E4122200E1
:103E00004C30EF01032F2000C70031009518052F1B
:103E1000151720004708310091007030920094017E
:103E200022006F083100930003108B1B03148B13C7
:103E3000151555309600AA309600951495181E2F2A
:103E4000151103188B170800B1002100200820006D
:103E5000B200210021082000B30021002208200028
:103E6000B4000800B100210023082000B2002100A6
:103E700024082000B300210025082000B400080019
:103E8000220055082000C400220056082000C5006A
:103E9000220057082000C600080041082200D50073
:103EA000200042082200D600200043082200D7004C
:103EB000080041082300E400200042082300E50038
:103EC000200043082300E600080022002608200006
:103ED000BB00220027082000BC0022002808200088
:103EE000BD007A08A03E8600013087000108080066
:103EF000C300230043082000C4002300440820001E
:103F0000C500230045082000C600080064082400FE
:103F1000BF00230065082400C000230066082400B9
:103F2000C10008007A35203E860003308700080073
:103F300041082300C300200042082300C4002000E1
:103F400043082300C50008002200E800E901E83525
:103F5000E90DE835E90D0800AE302000AF0007306C
:103F6000B0003F3414302000AF006E30B0003F345A
:103F700085302000AF006B30B0003E343D30200073
:103F8000AF008A30B0003F342F08C4003008C500AD
:103F90003108C60008002F08BE003008BF003108F5
:103FA000C0000800200062083F394038E2000800E5
:103FB000403F2400C800413FC9000800FF30B2065E
:103FC000B306B406B20A08006008F0390138E00010
:103FD0002200080020006208CF391038E2000800F3
:103FE00020006108FC390138E10008002000580871
:103FF0000339033A08002200B730EF01EF0A080046
:10400000FF3FFF3FFF3FFF3FFF3FFF3FFF3FFF3FC0
:10401000FF3FFF3FFF3FFF3FFF3FFF3FFF3FFF3FB0
:10402000FF3FFF3FFF3FFF3FFF3FFF3FFF3FFF3FA0
:10403000FF3F2000B4000130B7012200DC02003055
:10404000DD3B5C085D04031D5628DC01DC0ADD0154
:1040500021009D183F2820004D1B3F288E317A26D5
:10406000A0312F08B6002E08B5003608B300350879
:10407000B200B336B20CB336B20C3208B70020002F
:10408000531C542853109631E826A0312100D40146
:10409000D501200034082100C900FF302200DC00D7
:1040A0002F30DD000E14562822000E102000370895
:1040B000080054085504031961280130D402003067
:1040C000D53B22006608670403196A280130E6021E
:1040D0000030E73B200057197828023021003502D4
:1040E000D0300319340203187828B40A0319B50A2A
:1040F00020004E1A86281E3022004A02FF30031983
:10410000490203188628C90A0319CA0A21002C0883
:104110002D0403198F280130AC020030AD3B4D084F
:104120006D06031D98287F304C0203189828CC0A8E
:104130002200430844040319A1280130C3020030BF
:10414000C43B21002E082F040319AA280130AE0217
:104150000030AF3B2200470848040319B328013060
:10416000C7020030C83B450846040319BB2801308C
:10417000C5020030C63B410842040319C328013080
:10418000C1020030C23B6A086B040319CB2801301E
:10419000EA020030EB3B6C086D040319D3280130B0
:1041A000EC020030ED3B21006708031DE7033008F7
:1041B00031040319E2287308031DE2280130B0021C
:1041C0000030B13B5C080319F6282200640865043E
:1041D0000319EF280130E4020030E53BF628210006
:1041E000CD30DC032200E4000430E5002200620848
:1041F000630403190B2921002B0820005202031D20
:104200000329F327A03103180B2901302200E20211
:104210000030E33B08002200600861040319080035
:104220002000520821002B02031D19298F31C527B8
:10423000A0310318080001302200E0020030E13B09
:1042400008002000CE112100570B472992132800A7
:104250009501210062082800960008307202031CB4
:10426000392920004D1A3929720828001602073E04
:10427000960022000C108C102000CD1842293D0021
:10428000910144293D0090012000CE148129023083
:104290005706031D73298421A03120000330CE105E
:1042A00028009704950122004E082800960020005F
:1042B000640C0339013A031D612928001608F83EF1
:1042C000960020004D1E68292100630828009600F2
:1042D0002000CD186D2900306E2901308A21A031CF
:1042E00020001110812903305706031D8129280061
:1042F0001708FC390238970095012100D7012000EA
:10430000CE152100D70A08009D1808009D14200032
:104310004D130800F5007508031D90299727A0315B
:10432000750B08009E2708002000481808005E084A
:104330000339023A0319622BCD1CA2295E08033906
:104340000319A929CD18942A5E080339013A031DDF
:10435000942A22000E1CFF2920005415D418D229BB
:104360003D006527A031031DBA2922008E1CBA2901
:104370008C27A0315F27A031031DC32922000E1D09
:10438000C3298027A031DB27A031031DCB292200C0
:104390008E1DCB298627E0303D0092058A314322CD
:1043A000A031D829D627A0310319D829E023A0317C
:1043B000D627A031031DFF292000D41CFF2922008D
:1043C0000E102000620E0339023A031DE929220073
:1043D0008E105F27A031031DEF2922000E1120004F
:1043E0005E0E0F39093A031DF72922008E11FA26B5
:1043F000A0311C27A031611EFF29EA27A03122002D
:104400000E1C0C198A2A210026082704031D8A2A5B
:104410003D007727A031031D152A22008E18152A8A
:104420002000481F152A8C27A0315327A031031DD7
:10443000212A22000E19212A20004A1C212A802725
:10444000A031E027A031031D2D2A22008E192D2A2C
:104450002000C91E2D2A8627A031E023A031E527A0
:10446000A031031D802A2000D418802A21004E0884
:104470004F04031D802ABD27A031031D462A481F73
:10448000442A22008E14462A22008E105327A0317F
:10449000031D512A4A1C4F2A22000E15512A2200C0
:1044A0000E11E027A031031D5C2AC91E5A2A2200E2
:1044B0008E155C2A22008E11D826A0312000903063
:1044C00054114927A03103195D2B9227A031031DF8
:1044D0006E2AF4302100CE000130CF002000611E92
:1044E00008002C304927A031031D782A0830FC2F02
:1044F0004B0E890C0339023A031D08006430FC2F6F
:1045000021004E084F04031908000130CE0200308C
:10451000CF3B0800210026082704031908000130BA
:10452000A6020030A73B0800CD189A2A5E0803397E
:104530000319A12ACD1C08005E080339013A031DA6
:10454000080022000C1DF32A20005415D418CA2A92
:104550003D007727A031031DB22A22008E1CB22A0B
:104560008C27A0315327A031031DBB2A22000E1D2A
:10457000BB2A8027A031E027A031031DC32A2200D7
:104580008E1DC32A8627E0303D00A0058A314322D4
:10459000A031D02AE527A0310319D02AE023A03189
:1045A000E527A031031DF32A2000D41CF32AB127EC
:1045B000A031031DDD2A22008E105327A031031DD8
:1045C000E32A22000E1120005E0E0F390A3A031D65
:1045D000EB2A22008E11D826A0311C27A031611EA3
:1045E000F32AEA27A03122000C1D0E188A2A210086
:1045F00026082704031D8A2A3D006527A031031DD4
:10460000092B22008E18092B2000481F092B8C270C
:10461000A0315F27A031031D152B22000E19152B89
:1046200020004A1C152B8027A031DB27A031031D59
:10463000212B22008E19212B2000C91E212B862719
:10464000A031E023A031D627A031031D802A20000D
:10465000D418802A21004E084F04031D802A22000E
:104660000E142000620E0339023A031D3E2B481F30
:104670003C2B22008E143E2B22008E105F27A0318F
:10468000031D492B4A1C472B22000E15492B2200E3
:104690000E11DB27A031031D542BC91E522B220003
:1046A0008E15542B22008E11FA26A0312000903056
:1046B00054114927A031031D652A0A302100CE007C
:1046C000CF016E2A571C9D2BCD187D2B5415B12779
:1046D000A031031D722B5F1E702B22008E14722BD3
:1046E00022008E105327A031031D782B22000E11BB
:1046F00022000E14200054110800CD1C080054158F
:104700005E19852B22000E10982B620E0339023A97
:10471000031D922B5F1E8F2B22008E14982B2200DC
:104720008E10982BAC27A031031D982B22000E1160
:1047300022000C15200054110800CD18BB2B541575
:10474000BD27A031031DAB2B5F1EA92B22008E14A9
:10475000AB2B22008E105327A031031DB62B5F1EFA
:10476000B42B22000E15B62B22000E1122000E10C3
:10477000200054110800CD1C080054155E19C32BED
:1047800022000E14DB2B620E0339023A031DD02BDC
:104790005F1ECD2B22008E14DB2B22008E10DB2B14
:1047A000AC27A031031DDB2B5F1ED92B22000E1579
:1047B000DB2B22000E1122000C11200054110800E6
:1047C0002000D41C080021003708031D212CA03034
:1047D000250016020318EE2B960AF42BA0301606BD
:1047E000031DF42B2000D41021005E08F83EB70012
:1047F0008F312227A0310319571C072C21003708BD
:104800002000A7000530A926A0312100B7005927B4
:10481000A031031D0E2C2100B7361D2C9227A0318C
:10482000031D1D2C210037082000AA00AA36AA3635
:10483000AA362A0821003702B7002000611E0800AE
:10484000EF2FB703080020005419F12C5908720605
:10485000031D3D2C59085C020318322C590803191A
:10486000322CD9035C085902031CCD1B382CD90A01
:1048700059084327A0312100C900210049087306C7
:1048800003195F2C54085504031D5F2C2000CE181B
:104890005F2C9631E826A03197319627A031210070
:1048A00049088B316823A031F3007308031D5F2C86
:1048B0008E317326A031C125A0312000CF1273089C
:1048C00021004906031DD42C200053115908F20081
:1048D0001A307202031C762CB827A031BB35BC0DF0
:1048E000A527A0310318BC0ABF30AB2C14307202CC
:1048F000031C902C7208AF31F127A031AE31DE26B7
:10490000A03128082200BC00200027082200BB009C
:10491000210063082200BB070318BC0AD830AB2C67
:104920000F307202031C9C2CB827A031A527A031A0
:104930000318BC0AEB30AB2C08307202031CAF2CFE
:1049400072082200BB00BC01210063082200BB07E3
:104950000318BC0AF930BB07031CBC03B42C2100AC
:1049600063082200BB00BC0101303C020030031987
:104970003B02031CBE2CFF30BB00BC013B08CE0039
:1049800016307202031CC92C21005F082200D000DF
:10499000CA2CD00172082300E800E836E836E83671
:1049A0006808033C2200CF0072084327A031730639
:1049B0000319F12C2000590872020318E12C541B32
:1049C000E62C72085902031CD41EF12C7208D9007F
:1049D0004327A0312100C900200059353A27A031D2
:1049E000AB007308031D092D7208031D092D20005B
:1049F000CE1DFC2C210092102200E601E7012000D0
:104A0000CE108E317326A031CD15C125A0312000E6
:104A1000CF1205307302031C112D2100141A112D21
:104A2000141605307302031C252D21009218252D24
:104A3000200060080F39063A0319252D5F080F3949
:104A4000063A0319252D210092140530730203182C
:104A50002E2D2000CE1D2E2D21009210F827A031E2
:104A600003193506031D3A2D4808031D3A2D200071
:104A7000CA1E472D2100320F402D330A0319472D3E
:104A80002200490A1E3003194A06031D4A2D200040
:104A90004F144C2D20004F10FF3021003302003006
:104AA00003193202031C592D2000D9012100D40121
:104AB000D501A8303406023003193506031D762DC2
:104AC00048080319762D2000CA1A762DCA166208E6
:104AD0000F392300E80005306802031C762D2500FD
:104AE000A831F220A0319F310327A03120004D1AB8
:104AF000822DCB25A031063073020318882DC125E5
:104B0000A031882D21009218882D97317027A0316F
:104B100020004D1DAB2D2300210873020318932D97
:104B20002000C427A0317308031DAB2D20005B08B3
:104B3000031DAB2D7208031DAB2DCE10CD15963184
:104B4000E826A03120005419AB2DB526A0314D1117
:104B5000CD1FAB2DCD132000CD1CB02D0130B12DBC
:104B600000302300E80020004D1CB82D0130B92D85
:104B7000003023006806031D08002000541D4D115D
:104B800008002000DA012200D1012100B801200034
:104B9000DB01C427080072085902031CD12D7235AD
:104BA000DC2D720859020318DF2D72084327A0314B
:104BB00073020318DF2D59353A27A031AB000530B9
:104BC00073020318E92D2100AA01AB012000D101D5
:104BD000D201220062086304031D292E21002B0844
:104BE00020005202031DF62DF327A031031CCD1B1C
:104BF000292E4D19292ED10A0319D20ACA27A0310C
:104C0000A926A031AB00FC30A7004B0E890C03395C
:104C1000013EAC00003003180130AD002D0DAD0C8D
:104C2000AC0C2D0DAD0CAC0C2C08A9262B07AE003E
:104C3000210061082000AE020530A7007208AF31E4
:104C4000A527A0312E021A3EB1002200E200E301A6
:104C50009C2E220060086104031D9C2E2000520837
:104C600021002B02031D372E8F31C527A0310318D9
:104C70009C2E01302000D1020030D23BCD1F712E7E
:104C800015307202031C462EB1014E2E2200500830
:104C900021005F0222004F072000B10021002A08F6
:104CA000200051026E27A031153003192B02031C7E
:104CB000612E16307202031C612EEC30D107FF30DA
:104CC000D23D21002A08200051026E27A031213058
:104CD00003192B02031C982EF830D107FF30D23D68
:104CE000982E0930A7007208AF31A527A031AB007C
:104CF0004B0E890C0339AC00CA27A031013EAD0030
:104D0000003003180130AE002E0DAE0CAD0C2E0D90
:104D1000AE0CAD0C2D08A926A031AF002C082F0237
:104D2000B0002B08300221006007073E2000B100D0
:104D300031082200E000E1011E307202031C08006D
:104D400021002B082000D20021002A082000D100D9
:104D50000800A900A80127082918A807A735A9361F
:104D60002908031DAB2E28080800CE1808004D188E
:104D7000C92E9727A03121008E1623008E16210000
:104D80001D08033954389D000E1222000E12200017
:104D9000CD104D1C08009E27A031D0271D080339D7
:104DA00050389D008E1222008E122000CD14080073
:104DB00022000E10E0303D0092052000620E033903
:104DC000033A031DE62EE0303D00A1052000600EF1
:104DD000890C0339033A031DF02EE0303D00A20593
:104DE00020005E0E0F390A3A031D0800E0303D0036
:104DF000A305080022000C11E0303D00A0052000B2
:104E0000620E0339023A031D082FE0303D00A10570
:104E10002000600E890C0339023A031D122FE03086
:104E20003D00A20520005E0E0F39093A031D08005F
:104E3000E0303D00A305080080302100A6000C30C2
:104E4000A70020004B0E890C0339033A031D2D2FB8
:104E5000F4302100A6000130372F4B0E890C0339A6
:104E6000023A031D382FF0302100A6000A30A700B7
:104E700020000800A03E860002308700403F21004D
:104E8000AA00413F0800A03E8600013087000108CB
:104E900008002100CE000130CF0020004B0E890C0D
:104EA0000339033A08002000600E890C0339033AE5
:104EB000080020004B0E890C0339033A080020003B
:104EC000600E890C0339023A08002008E0390D38D9
:104ED000A0002000620E0339023A0800AB00210056
:104EE0002B082000523BAC0000302C0208001208B6
:104EF000E0390D3892002000620E0339033A0800B1
:104F00003D002208E0390D38A20008003D002308CA
:104F1000E0390D38A30008003D002108E0390D38C4
:104F2000A10008004B0E890C0339023A0800220048
:104F30000C143D00900102309100080022008C14F6
:104F40003D009101023090000800BB35BC0D2100EE
:104F500063082200BB070800600E890C0339023A7F
:104F6000080022000C112000620E0339033A0800E9
:104F700072082200BB00BC01080022000C152000B2
:104F8000620E0339033A0800D101D2012100AA01BF
:104F9000AB010800FE30A7004B0E890C0339080056
:104FA00021000E1623000E16210008003D002008E7
:104FB0001F390D3A080020005E0E0F39093A08002B
:104FC00020005E0E0F390A3A08003D0012081F3912
:104FD0000D3A0800C8302100A600A70108002100F2
:104FE000B701B70A080021002A0820005102080072
:104FF000D0302100340602342100CE00CF01080059
:10500000FF3FFF3FFF3FFF3FFF3FFF3FFF3FFF3FB0
:10501000FF3FFF3FFF3F4C062000E200620E08000A
:105020002000620E890C890C08002400CC00CC0EF4
:10503000CC0DCC0D20000800890C01392400CF00D4
:1050400020000800200060089F392038E000080098
:1050500001392400CC007408CD0008002400CD00E4
:10506000CD0C4D0C0139CE002000080024004C0668
:10507000FE394C06200008002400CC00CC0ECC0DDC
:1050800020000800F436F4367408073908000730A9
:105090007405CC00063A080007307405CC00053AC8
:1050A00008004E074D074C072100C40720000800E8
:1050B0004C06CE00CE0DCE0DCE0D200008000330E4
:1050C000F436F4367405CC00033A080050074F0755
:1050D0004E074C072100C400080007307405CC00BF
:1050E000033A08002000580803392400CC00733428
:1050F00007307405CC00073A080007307405CC006F
:10510000023A0800890C01392400CE002000080072
:105110006610E6106611E6116810080024004C06BF
:10512000BF394C062000080071082400CC00CC0ECA
:1051300020000800890C890C01392400CC000800EB
:1051400020004D15DC01D412541708005A302200FB
:10515000EF00523424004C069F394C062000080012
:105160002000C90074082400CC00080024004E066A
:10517000F7394E06200008006612E6126613671320
:10518000E71308004B0E890C03392400CC000800FB
:10519000640C03392200EF00433407307405CC005F
:1051A000043A080003307405CC00023A08002200DB
:1051B000B330EF01EF0A08002100470820005D0628
:1051C00008005A302200EF0040344B0E890C03399E
:1051D000013A0800FF302200EF00A0345A302200CC
:1051E000EF00423412082200EF00A8342300210807
:1051F00073020318062920005C08031D06295B08BA
:1052000003190329DB035A08031DDA012000CE1815
:1052100008005A08A000A10173085B07A200A301BF
:10522000A30D20082207A4002108233DA500803AF1
:10523000A60080302602031D1F29C1302402031C52
:105240002229DE2FA03020001E06031D2D29063046
:10525000F50073084021A8313C2980301E06031D4B
:1052600037290330F50073084021A8313C2960300C
:105270001E06031D3E29733673023F297308D02F83
:10528000F600F801750803195629F701F70AF51B0E
:105290004B29F5354629F83575087602031C532944
:1052A0007508F6027814F536F70B4B2978080800D4
:1052B00062080F39013A0319622962080F39043A6A
:1052C000031D972962080F39013A031D6A29CA1D77
:1052D000F629F32962080F39043A031DC62A220071
:1052E0006A086B04031D7C292000CA1D7A2922004C
:1052F0008E147C2922008E107308031DC62A2000FC
:105300004E18CD1FC62A21004A08031DC62A0030A8
:105310002D028D3003192C020318C62A22008E1488
:105320000C30EA00EB012100CA01CA0AC62A620851
:105330000F39023A031DF9294A1ECA1DA12940301E
:10534000C806DE22A831620E0339013A031DAC29DA
:10535000F522A8310319F129620E0339013A031D20
:10536000DC29FB22A831031DCB295C080319C229C3
:10537000481FBD2922008E14BF2922008E10C82488
:10538000A831C62A7308031DC62A2100300831043B
:10539000031DC62AF6290123A831031DC62A5C086D
:1053A000031DBD297308031DC62A210030083104DE
:1053B000031DC62A2000F129F522A831031DC62AA3
:1053C000620E0339023A031DE929CD1C5419C62A7D
:1053D000F129620E0339033A0319CD1CC62A541968
:1053E000C62A481FF62922008E14C62A22008E10D3
:1053F000C62A62080F39033A031D542A4A1ECA1DE1
:10540000022AC914DE22A831C91C512A250012081B
:10541000031D252A22008E10EF22A83121006C08DE
:105420002500920021006B082200C300C401210066
:105430006B08AE00F030AF01AE0EAF0EAF052E0818
:105440000F39AF04F030AE05C62A220043084404E9
:10545000031D352A2500120821006C06031D352A7C
:105460006C36CB0025009200C62A003021002F02A6
:10547000213003192E020318C62A25001208210024
:105480004B06031DC62A2E082F0403194A2A2200A0
:105490008E14832A250092010723A8312000C91009
:1054A000C62A25009201812A62080F39053A031D98
:1054B0005C2ACA19892A812A62080F39063A031D13
:1054C000922A4A1ECA1D662A4030C806DE22A8312A
:1054D000F522A831031D6F2A481B892A812AFB2245
:1054E000A831031D782A7308031D481F812A872AC3
:1054F0000123A831031DC62A5C08031D812A481B0D
:10550000872A22008E10E0303D00A105C62A481FE0
:10551000C62AA8309531E325A83125009200EF2254
:10552000A831C62A62080F39073A031DC62A21008E
:105530006708031DC62A20004A1ECA1DA12A103072
:10554000C806DE22A831CA1DC32A481AB52AA230CD
:10555000250012020318B52A21006708031DB52A89
:10556000EF22A8312500920AC32A2000481EC32A30
:1055700021006708031DC32A250012080319C22A47
:105580009203C32A07230C302100E7002000480EB5
:10559000890C890C01392300E800A4309531E325FA
:1055A000A831230068060319080000302000481BBA
:1055B00001302200EF00A4309F31032F4A0C23005A
:1055C000E800E80C680C0139E900E90E20004A08FF
:1055D00023006906EF3969062000CA0008003D0073
:1055E0002108E0390C38A1000800620E890C890CF2
:1055F0000339013A0800620E890C890C0339023A1A
:105600000800620E890C890C0339033A0800220055
:105610008E10E0303D00A1050800CE24A831031D06
:10562000692BD324A831031D1A2B61080339013AD1
:1056300003195A2BD324A831031D4D2B61080339BC
:10564000023A031D362B7308031D2B2B2100300853
:1056500031040319A42B20005C080319782C4A1884
:10566000402B22000E11C824A831782C6108033980
:10567000033A031D782C5C080319432B4A1D312B78
:1056800022000E15332B7308031D782C21003008DF
:105690003104031D782C2000662B61080339013A80
:1056A000031D782CA731AC27A831031D5D2BCD1C21
:1056B0005419782C4A18A72BAA2B600E890C033991
:1056C000033A0319CD1C782C5419782C4A1CAA2BA8
:1056D000A72B60080F39023A031DAD2BCA1C722B91
:1056E0000130732B0030AD004A1C782B0130792B30
:1056F00000302D0603199F2B4A0C890C0139013CFF
:10570000AD00AD0DAD0D22000E0820002D06FB39B9
:105710002D0622008E0021006F082000A7003130E6
:10572000A801A900AA01DE26A83128082200ED0060
:10573000200027082200EC002000B824A831220015
:105740006C086D04031D782C20004A1DAA2B220032
:105750000E15782C22000E11782C60080F39033AB0
:1057600003195F1A092CCA1CB72B0130B82B003063
:10577000AD004A1CBD2B0130BE2B00302D06031995
:10578000C42B4914B824A831491C2A2C260012081D
:10579000031DE62B22000E11C224A83121006C0843
:1057A0002600920021006B082200C700C8012100DA
:1057B0006B082200C500F030C601C50EC60EC60536
:1057C00045080F39C604F030C505782C220047087B
:1057D0004804031DF42B2600120821006C06031D4B
:1057E000F42B6C36CB00272C0030220046022130EF
:1057F000031945020318782C2600120821004B06D5
:10580000031D782C2E082F04031D562C2000491050
:105810002A2C60080F39043A031D5C2C571C122CEB
:105820005F1A142C5F1A2F2C4A1C2A2C22000E15EA
:10583000C224A83120005A08AD00AD36AD36AD36D1
:105840005B352D0773079C24A83168086A0726007A
:105850009200782C2600920122000E11582C5F1A1B
:105860005718782C4A18532C22000E1120005A0881
:10587000AD000430AD36890B3A2C7308AE00AE365D
:105880005B352E072D079C24A8316803FF3A2000C2
:10589000AD0021006A0820002D02A03E26009200E3
:1058A000C224A831782CA0302600920022000E15C8
:1058B000E0303D00A205782C60080F39053A031D41
:1058C0006B2C4A080139AD00AD0E4B082D06EF399F
:1058D0002D06CB00782C60080F39063A031D782C72
:1058E000CE194A1C762C21009210782C210092149B
:1058F000200060080F39013A0319832C60080F3922
:10590000043A031D080061194E1808007308031DAE
:1059100008005F1E8E2C5F1A571C932C22000E115C
:105920002600920108005F1A5718080022000E1581
:10593000A0302600920008002100EA0069080A3E13
:105940002000AD00003003180130AE00803AAF00F7
:1059500080302F02031DB02C21006A0820002D0288
:105960000318B62C210069080A3EEA00210008004D
:105970004A080139AD00AD0D4A082D06FD392D0646
:10598000CA0008003D002208E0390E38A2000800D5
:105990007E302100B0000230B10008002000600815
:1059A0000F39013A0800600E890C0339013A0800EA
:1059B0002300210873020318E82C20005C08031D53
:1059C000E82C5B080319E52CDB035A08031DDA01F8
:1059D0002000CE1808005A08AB00AC0173085B0722
:1059E000AD00AE01AE0D2B082D07AF002C082E3DEB
:1059F000B000803AB10080303102031D012DC1306A
:105A00002F02031C042DDE2FA03020001E06031DD4
:105A10000F2D0630A7007308A527A8311E2D803052
:105A20001E06031D192D0330A7007308A527A831F2
:105A30001E2D60301E06031D202D73367302212D8E
:105A40007308D02FB4302200CB0023082000C100FF
:105A5000220024082000C200220025082000C300E4
:105A6000B43096316B26A831E4279531F525A8315D
:105A700041082200A000200042082200A1002000CE
:105A800043082200A200230021087302031C792D81
:105A9000220020082000B600220021082000B700C4
:105AA000220022082000B800B231E222A831B2312F
:105AB0001F22A831B231D022A8319C31A824A831AC
:105AC00064082200D10005307202031C6F2D2100F2
:105AD000650A22006C2DD136890B6B2D792D2100A2
:105AE00066082000A70022005108A527A83122003F
:105AF000D1002000D31CA22D220022082104200462
:105B00000319A12D20008030BB01BC003F30BD0037
:105B1000220020082000BE00220021082000BF0033
:105B2000220022082000C0009C318D243B08220066
:105B3000A00020003C082200A10020003D08220017
:105B4000A200D101220051082100B800080070080D
:105B500003392400D70051309531E325A8312400C2
:105B600057060319B52DFF30C82D70080339D7002B
:105B700051309531E325A83124005706031DCE2D61
:105B800050309531E325A8315A3A0319CE2D5A30B9
:105B90002200EF0050309F310327A831EB279531C9
:105BA000E325A831240057060319D82DFF30E82D2E
:105BB000EB279531E325A83124005706031DEE2D70
:105BC00054309531E325A8315A3A0319EE2D5A3055
:105BD0002200EF0054309F310327A8316430953103
:105BE000E325A831003A031DFB2D9731C427A831C6
:105BF0009F310327A8314B309531E325A831013A75
:105C0000031D072E013090311E20A831092E0C26CD
:105C1000A831F3269831772850309531E325A83103
:105C20005A3A031D812E52309531E325A8315A3A54
:105C3000031D812E54309531E325A8315A3A031DB6
:105C4000812E55309531E325A831003A0319372EBE
:105C500055309531E325A8312400C8000F304802A3
:105C60000318372E55309531E325A831382E0230F0
:105C70002500A200A301023E2100D6000230FA0056
:105C80001F307A020318C92E7A08543E9531E32555
:105C9000A83196316B26A831E42723006A0820003A
:105CA000C10023006B082000C20023006C08200004
:105CB000C3009531F525A8319F315927A8319C3172
:105CC000A824A831BE27A8316408C03F6508C13F99
:105CD000D827A8317A35A03E8600403FCA00413F10
:105CE000CB0049084B02031D772E48084A020318CF
:105CF0007F2ED827A831BE27A831F727A831FA0A66
:105D0000402EFA012030FA0A7A020318B82E7008E1
:105D10000339023A031D992E7A082000F127A83191
:105D2000DE26A831BE27A8312708C03F2808C13F7A
:105D3000A42E7A082400C800C901C835C90DC83589
:105D4000C90DBE27A831F7279F31F627A831031DBB
:105D5000822EBE27A831403F2400C800413FC90021
:105D6000C936C80C7A35A03E8600F727A831822EA6
:105D700052309531E325A8315A3A0319C92EA8317A
:105D8000A620A8319F310327A831FC279F31032784
:105D9000A83125000030A001A1015D02E8300319FF
:105DA0005C020318DA2E5C08183EDE0000305D3D10
:105DB000DF000800FF30DE00DF010800AB01AC01AE
:105DC000271CE62E2908AB072A08AC3DA935AA0DE9
:105DD000A836A70C27082804031DE02E2C08A800CD
:105DE0002B08A70008002300A00120004D1A272F30
:105DF00053309531E325A8312300A1000230FA0089
:105E000020307A020318272F7A08A03E860001303E
:105E100087007A081F3E84000230850000082000B9
:105E2000AB007A089F3E84000130850000082B07F4
:105E300081007A08A03E8600C3300102031C252F92
:105E40007A08A03E8600C2308100FA0A002F2000A6
:105E50004D1AD41D782F70080339023A0319522FB6
:105E6000FA011730FA0A7A0203183F2F7A08A03E87
:105E70008600013087007A08043E8100312F1C30F3
:105E80002300B7001E30B8002130B9001A30FA00E4
:105E900020307A020318782F7A08A03EC427A83150
:105EA000FA0A482F70080339023A031D782FFA01C5
:105EB0001530FA0A7A020318662F7A08A03E860087
:105EC000013087007A08083E8100582F21302300D6
:105ED000B5001630FA0020307A020318782F7A08BD
:105EE000A03EC427A8312030FA0A7A02031C6F2F83
:105EF00021002030BA01B901FA007A08031908001C
:105F0000A03E86000130870003302000A700230058
:105F10003F08A527A83101027A08031C922F21000F
:105F2000BA007A08A03E86000130870023003F08AF
:105F30002000AB00AB36AB362B080102031CA32FAD
:105F40007A082100B900FA037D2F2000A800AA01D9
:105F500027080319BC2FA901A90AA71BB12FA73530
:105F6000AC2FAA3527082802031CB92F2708A8023E
:105F70002A14A736A90BB12F2A0808007A35A03EAB
:105F800086000230870008008600013087007A080A
:105F90009F3E8400013085000008043E8100080017
:105FA0002100B60020005B075A072C00980008006B
:105FB000210056082400C800C901080020001E085E
:105FC000023E2C00980008002F08C4003008C500CD
:105FD0003108C60008002000580803392400D70003
:105FE0007334A7000330A801A900AA0108004808DB
:105FF000C03F4908C13F08000C302200EF00533475
:10600000FF3FFF3FFF3FFF3FFF3FFF3FFF3FFF3FA0
:10601000FF3FFF3FFF3FFF3FFF3FFF3FFF3FFF3F90
:10602000FF3FFF3FFF3FFF3FFF3FFF3FFF3FFF3F80
:10603000FF3FFF3FFF3FFF3FFF3FFF3FFF3FFF3F70
:10604000FF3FFF3FFF3FFF3FFF3FFF3FFF3FFF3F60
:10605000FF3FFF3FFF3FFF3FFF3FFF3FFF3FFF3F50
:10606000FF3FFF3FFF3FFF3FFF3FFF3FFF3FFF3F40
:10607000FF3FFF3FFF3FFF3FFF3FFF3FFF3FFF3F30
:10608000FF3FFF3FFF3FFF3FFF3FFF3FFF3FFF3F20
:10609000FF3FFF3FFF3FFF3FFF3FFF3FFF3FFF3F10
:1060A000FF3FFF3FFF3FFF3FFF3FFF3FFF3FFF3F00
:1060B000FF3FFF3FFF3FFF3FFF3FFF3FFF3FFF3FF0
:1060C000FF3FFF3FFF3FFF3FFF3FFF3FFF3FFF3FE0
:1060D000FF3FFF3FFF3FFF3FFF3FFF3FFF3FFF3FD0
:1060E000FF3FFF3FFF3FFF3FFF3FFF3FFF3FFF3FC0
:1060F000FF3FFF3FFF3FFF3FFF3FFF3F430852028D
:10610000031D842842085102031CA028D310520802
:10611000A8005108A7004208A7024308A83B643022
:10612000A900AA01AE31DE26B031ED228D31E7257E
:10613000B0312F08C5003008C6003108C700A428B8
:10614000D314C501C601C701510852040319C92857
:106150005208B0005108AF008D31E725B0312F084B
:10616000B3003008B4003108B5004508B600460851
:10617000B7004708B8001F22B03133082200A3003F
:10618000200034082200A400200035082200A500C9
:10619000CB28E822B031200051085204031DD12839
:1061A000E82220004508C2004608C3004708C40092
:1061B0000800210049080319062A2000D31FD2290C
:1061C000210038082400C800C901C809C909C80A43
:1061D0000319C90A4908CB0073084802CA00031C06
:1061E000CB03C23ECC0000304B3DCD00803ACE0008
:1061F00080304E02031D002920005B0824004C0261
:10620000031CD22973080319D22906302000AF00DD
:10621000B0014B0E890C03392400C800C901C835F0
:10622000C90D48082000AF02240049082000B03BF7
:10623000AF35B00DAF35B00D7C22B0312F08B300B3
:106240003008B4003108B500220023082000B60051
:10625000220024082000B700220025082000B800F2
:106260001F22B03133082200D2002000340822005F
:10627000D300200035082200D4005A085B04031D17
:10628000C8292000DB0ADC22B0317208DA070318C3
:10629000DB0AFB30DA07031CDB037308230024024C
:1062A000031C5C29730821004902031C5C2920009F
:1062B0005412DC22B0315E29200054162000B401B3
:1062C000B501B601220052082000B7002200530891
:1062D0002000B800220054082000B9009822B031F4
:1062E000031C541EBD2922005B082000A8002200C8
:1062F0005A082000A7006430A900AA01AE31DE26AA
:10630000B031ED228D31E725B0312F082300C000D8
:10631000200030082300C100200031082300C20003
:10632000220052082000B300220053082000B400CD
:10633000220054082000B5002300C422B0311F22DF
:10634000B03133082300C000200034082300C1000E
:10635000200035082300C200C422B031E222B0314F
:106360001F22B031D0229C31A824B0316508220010
:10637000DB00230064082200DA00720820005C02BF
:106380000318CC292200DA35DB0DDA35DB0DCC29F8
:106390000130DA020030DB3B2000D3132200D801A9
:1063A000D80AD9012000541C062A5B080319062AC2
:1063B0005410220058085904031D022A09302000F5
:1063C0005B020318FB2904302200D8000730D901F2
:1063D0002000A7007208AF31A527B0312400C80003
:1063E0002200D802031CD903D835D90DD835D90DD0
:1063F000D80A0319D90A21003808031DB803200060
:10640000DB03062A0130D8020030D93B7308200094
:106410005B072400C800C901C90D4908803A803CC7
:10642000031D152A48082300210203180800230031
:1064300021087302031808002000DB010800360859
:10644000B9003708BA003808BB0003103A0D3B0DFD
:10645000C0004008031D2D2AF22A3308B900340871
:10646000BA003508BB0003103A0D3B0DC1004108CE
:10647000031D3B2AF22A8930BD01BE01BF0141073D
:10648000B900C0023808C1003508C1068030C10516
:106490001830B717B801B417B501BC00BD35BE0D33
:1064A000BF0D35083802031D5B2A34083702031D6F
:1064B0005B2A33083602031C642A3308B602340808
:1064C000B73B3508B83B3D14B635B70DB80DBC0B1E
:1064D0004E2A3D08A7003E08A8003F08A900400832
:1064E000AA004108AB009631AA262708B300280865
:1064F000B4002908B5000800B201B01F862AAF0910
:10650000B009AF0A0319B00AB201B20A2F08A700F6
:106510003008A8008E30A901AA003208AB009631DD
:10652000AA262708AF002808B0002908B1000800F3
:10653000B61FA72A3408003CB4003508031C350FE9
:10654000003CB5003608031C360F803CB600B91F6E
:10655000B62A3708003CB7003808031C380F003C47
:10656000B8003908031C390F803CB9008030B606EA
:10657000B90639083602031D080038083502031D24
:10658000080037083402080040082000B600230045
:1065900041082000B700230042082000B80008008E
:1065A00033082300E400200034082300E500200025
:1065B00035082300E6000800210064082200DA0004
:1065C000DB010800C830B301B4004230B500080058
:1065D0002200A301A401A50108002808B000270893
:1065E000AF000800B301B401B5010800E51F0B2B93
:1065F00015307102031CFE2A1430F10071082500C9
:10660000A200A30171082200EF0055309F3103273B
:10661000B2318031F728671EFD2B07307102031855
:106620005E2B60087106F0397106E00071082200E7
:10663000EF00B1309F310327B2315A302200EF0012
:10664000B0309F310327B231AC31CE24B2310319BF
:106650005C2B33309531E325B2315A3A031D372B89
:1066600034309531E325B2312100EF003A2B21007F
:10667000EF01EF0AA8312220B2316108FC3901385C
:10668000E10060080F39043A03194D2B6111220013
:10669000B530EF019F310327B231A831D720B23195
:1066A0009F310327B2319F31FB27B2319F3103273E
:1066B000B231B7314227B2318131D8290B30710262
:1066C0000318932B08307102031C932BF930F10748
:1066D0007108A8313C20B2316008A831AA20B2313B
:1066E000E000600E890C87314027B231031C822BF9
:1066F0002000610887314027B231031C822B9F3173
:10670000F027B23171082200EF00B3309F31032728
:10671000B2315A302200EF00B2309F310327B2313C
:106720002200B730AC2C0D3071020318B12B0B30A6
:106730007102031CB12BF530F107710801396111A9
:10674000031D61150030611901302200EF00B530E2
:106750009F310327B2315A302200EF00B43081312B
:10676000D529103071020318E22B0D307102031C81
:10677000E22BF430F10761087106FC397106E10083
:10678000600E890C87314027B231031CD12B2000C9
:10679000610887314027B231031CD12BA831222058
:1067A000B23171082200EF00B7309F310327B231B8
:1067B0005A302200EF00B6309F310327B231220059
:1067C000B330AC2C1230710203185C2B1030710204
:1067D000031C5C2BF030F107710801396012031DB6
:1067E000601671082200EF00B9309F310327B231E3
:1067F0005A302200EF00B830AF2BE71ECA2C083009
:1068000071020318422C62087106F0397106E20029
:1068100071082200EF00C1309F310327B2315A3096
:106820002200EF00C0309F310327B2312000620800
:106830000F39053A0319212C62080F39063A031D56
:106840002F2CA8309531E325B2312500120603190B
:106850002F2CA831F220B2319F310327B231200012
:1068600062080F39073A031D372C250092012000DA
:1068700062080F39023A03195C2B6208CF391038CD
:10688000E200AA2C0B3071020318772C0830710239
:10689000031C772CF930F107A8319420B23162083B
:1068A00024004C06CF39A8310B20B2318731402764
:1068B000B231031C662CA8311020B2318731402739
:1068C000B231031C662C9F31D227B23171082200ED
:1068D000EF00C3309F310327B2315A302200EF005E
:1068E000C2309F310327B2312200C530AC2C0E30AC
:1068F00071020318AF2C0B307102031CAF2CF63061
:10690000F1077108A8311520B231620824004C0645
:106910003F39A8310B20B23187314027B231031CF7
:106920009C2CA8311020B23187314027B231031C92
:106930009C2C9F31EA27B23171082200EF00C5304C
:106940009F310327B2315A302200EF00C4309F310B
:106950000327B2312200C330EF01EF0AAF2B103012
:10696000710203185C2B0E307102031C5C2BF23099
:10697000F107710801396310031D631471082200C7
:10698000EF00C7309F310327B2315A302200EF00A9
:10699000C630AF2B671D012D0B3071020318E62C9A
:1069A000A8319420B2315E0824004C060F394C0601
:1069B0002000DE0071082200EF00D5309F31032750
:1069C000B2315A302200EF00D430AF2B10307102B8
:1069D00003185C2B0E307102031C5C2BF230F107A4
:1069E000710801396311031D631571082200EF005E
:1069F000D3309F310327B2315A302200EF00D2301A
:106A0000AF2BE71D332D073071020318182D5F08D7
:106A10007106F0397106DF0071082200EF00D730EF
:106A20009F310327B2315A302200EF00D630AF2B0E
:106A30001030710203185C2B0E307102031C5C2BAA
:106A4000F230F10771080139E311031DE3157108F4
:106A50002200EF00D9309F310327B2315A30220093
:106A6000EF00D830AF2B661C542D80307102031C10
:106A70003B2D7F30F100053071020318432D0430A7
:106A80006116F100482D71352100DE0020006112F1
:106A900071082200EF003D309F310327B2315A3098
:106AA0002200EF003C30AF2BE61C702D0530710248
:106AB000031C5C2D0430F10071082100DD00710819
:106AC0002200EF0041309F310327B231A831E1208D
:106AD000B2319F310327B23196317B26B2315C2B24
:106AE00080315A28D8259D310C25B531403095315B
:106AF000E325B5315A3A031D822D41309531E32506
:106B0000B531832D04302100DD0042309531E3257D
:106B1000B5315A3A031D9C2D43309531E325B531EB
:106B20002400D800D80D2000640824005806F93944
:106B300058062000E4009F2DF9302000E405352799
:106B4000B5313C000F10FF25B5316E27B53120005F
:106B50009210C825B531D425270091159215923190
:106B60004122B5317D26AD31A725B5310026210062
:106B700092141114141600309531E325B531D53A2D
:106B800003190800D5302200EF0000309F31032F99
:106B9000A33021009E00E0309F0583302200970043
:106BA000553021009D0008008B1710160B170800A8
:106BB0008E1623008E16A731D027B5318C162300F0
:106BC0008C1221000C1122000C1121000E10220049
:106BD0000E1021008E1022008E1021000E112200B6
:106BE0000E1121008E1122008E1121000C122200A4
:106BF0000C1224000C1621000C108C10FC2F802F7E
:106C0000200060304D11CD114D12CD124D17CE1018
:106C10004E124F104B11E3115E114816C911491263
:106C20004A12CA114913CA104A104910C910CB049C
:106C3000A4304D10CD1068125310D310D31354103C
:106C4000D4115411531561129531E325B531B12793
:106C5000B531031C322E2200A430EF019F310327EF
:106C6000B531432EA4309531E325B5312300E8003A
:106C7000E80EE80DE80D2000480823006806BF393B
:106C800068062000C800A9309531E325B531B12749
:106C9000B531031C522E2200A930EF019F3103278A
:106CA000B531622EA9309531E325B5312300E800D6
:106CB000E80EE80D2000490823006806DF39680661
:106CC0002000C900A7309531E325B531B127B53192
:106CD000031C6F2E2200A730EF019F31032FA73036
:106CE0009531E3252300E8002000480823006806CA
:106CF000FE3968062000C800080020005808033943
:106D0000031D9E2E73309531E325B5315A3A031D8C
:106D10008F2E76309531E325B531FF3E902E05302C
:106D20002100D8001F30FA01FA0A7A02031808007D
:106D3000AB27B531580881001F30942E580803390D
:106D4000023A031DCE2EFA010930FA0A7A0203181C
:106D5000AF2EAB27B531210058368100A42E093063
:106D6000FA0013307A020318C02EAB27B531210088
:106D70005808FF3E81001330FA0A7A02031CB52E30
:106D80001330FA001F307A0203180800AB27B53120
:106D900021005808033E8100FA0AC22E5808033920
:106DA000013A031DFE2E24000230A101A10AA20017
:106DB000A300A400A5000330A600A700A800A90016
:106DC0000430AA00AB00AC000530AD00AE000630C8
:106DD000AF00B000B1000730B200B300B40008301B
:106DE000B500B600B7000930B800B900BA000A30E3
:106DF000BB00BC000B30BD00BE00080058080339C2
:106E0000033A031D0800FA010730FA0A7A02031850
:106E10000E2FAB27B5318101810A042F0730FA000C
:106E20000E307A0203181C2FAB27B53181000E30CB
:106E3000FA0A7A02031C142F0E30FA0019307A0273
:106E400003182B2FAB27B531033081001930FA0A14
:106E50007A02031C222F04302400B900BA00BB00C0
:106E60000530BC00BD00BE0008005A27B5316627BA
:106E7000B531422796317B26B5316027B5318A2757
:106E8000B531912F2000921328001E15FC309E056D
:106E900020005F1E532F60080F39043A031D532F43
:106EA000033028009E04873028009E05A0309D00F6
:106EB0009C0108008030970046309800950108003A
:106EC00051309B009C0199019A01080092107E307C
:106ED00028009700FF309600950108007327B53110
:106EE0009727B531A02F250097170F309704171655
:106EF0000C309F04FF30960095012000D41008004C
:106F00002C00991719161F08FC3901389F009801A9
:106F100097010800413028009300940191019201EB
:106F2000080021309A009B01980199010800250072
:106F300093170F309304131603309F049201080037
:106F4000260093170F3093041316303025009F044A
:106F50002600920108007A08203E86000230870051
:106F600008002300E8000230680208005D082100E4
:106F7000CD003F30CD052000CF1FC12F4030210074
:106F8000CD0701309531E325B5315A3A031DCD2F98
:106F900002309531E325B531CE2F3D302100ED0093
:106FA0004D06031DD62F2000CA1EE32F21004D08D9
:106FB0006D06031DEF2F2000CA1EEF2F4030210069
:106FC0004C02031CEF2F20005715CA12F627B531CB
:106FD0002200C901CA01F22720004F10080020003A
:106FE000571108002000CE180800FC2F2100B40122
:106FF000B501B201B301080022000C148C14080082
:10700000FF3FFF3FFF3FFF3FFF3FFF3FFF3FFF3F90
:10701000FF3FFF3FFF3FFF3FFF3FFF3FFF3FFF3F80
:10702000FF3FFF3FFF3FFF3FFF3FFF3FFF3FFF3F70
:10703000FF3FFF3FFF3FFF3FFF3FFF3FFF3FFF3F60
:10743000FF3FFF3FFF3FFF3F1D309531E325BA314E
:107440005A3A031D282A1E309531E325BA313E2AC7
:1074500070080339013A031D2F2A03303E2A7008B1
:107460000339023A031D382A2100E501E50A402AC2
:1074700070080339033A031D402A04302100E50057
:107480001F309531E325BA315A3A031D4C2A20307A
:107490009531E325BA31602A70080339013A031D9A
:1074A000532A0430602A70080339023A031D5A2A0D
:1074B0000330602A70080339033A031D622A14302E
:1074C0002100E60021309531E325BA315A3A031DF7
:1074D0006E2A22309531E325BA31802A70080339AB
:1074E000013A031D752A0530802A70080339023AD3
:1074F0000319732A70080339033A031D822A0930DD
:107500002100E40023309531E325BA315A3A031DB6
:107510008E2A24309531E325BA31A22A7008033926
:10752000013A031D952A1E30A22A70080339023A37
:10753000031D9C2A1A30A22A70080339033A031D3E
:10754000A42A20302100E30025309531E325BA310B
:107550005A3A031DB02A26309531E325BA31B12AB3
:107560003D302100E20027309531E325BA315A3A07
:10757000031DC42A28309531E325BA3196316B2694
:10758000BA310C23BA31C92A23002030EA01EB00BA
:107590004230EC0087313827BA31F3229531F52596
:1075A000BA31002329309531E325BA315A3A031D07
:1075B000EB2A2A309531E325BA312100E1002B3046
:1075C0009531E325BA312100E0002C309531E325D7
:1075D0002100DF00080008302100E1000430E00055
:1075E000DF01DF0A080023006A082000C40023002E
:1075F0006B082000C50023006C082000C6000800AE
:1076000041082300EA00200042082300EB0020008C
:1076100043082300EC0008002F082300EA002000A4
:1076200030082300EB002000310823000800E51C8F
:10763000472B2930710203182D2B71082100E60019
:1076400066082200EF0020309F310327BB315A30FB
:107650002200EF001F308131D52929307102031C2F
:10766000C32B81307102031C372B8030F10071086D
:10767000D83E2100E50065082200EF001E309F3152
:107680000327BB315A302200EF001D302B2B651D24
:107690005E2B0530710203184F2B0530F100710885
:1076A0002100E40071082200EF0022309F310327FF
:1076B000BB315A302200EF0021302B2BE51D752BFA
:1076C0000A3071020318662B0A30F100710821009C
:1076D000E30071082200EF0024309F310327BB3103
:1076E0005A302200EF0023302B2B651E962B0730DB
:1076F000710203187D2B0730F10051307102031C19
:10770000832B5030F100710871077107013EF100C1
:107710002100E20071082200EF0026309F3103278C
:10772000BB315A302200EF0025302B2BE51EC52B34
:107730003D307102031C9E2B3C30F10071089631E4
:107740006B26BB31BB310C23BB31EC0087313827B2
:10775000BB31BA31F322BB319531F525BB31BB3199
:107760000023BB3171082200EF0028309F3103272E
:10777000BB315A302200EF0027309F310327BB3145
:10778000AE310C26BB318131D829651F212C0B303D
:1077900071020318CF2B71082100E100E82B15308E
:1077A00071020318DC2B0B307102031CDC2B7108F7
:1077B000F63E2100E000E82B333071020318E82B7D
:1077C00015307102031CE82B7108EC3E2100DF002C
:1077D0002A309531E325BB31210061060319F72BCF
:1077E00061082200EF002A309F310327BB312B3084
:1077F0009531E325BB31210060060319062C600892
:107800002200EF002B309F310327BB312C30953104
:10781000E325BB3121005F060319152C5F08220008
:10782000EF002C309F310327BB3129309531E32500
:10783000BB315A3A0319C32B5A302200EF002930CA
:107840002B2BB231F62A87316F27BC314C08F1005F
:107850002000A7319227BC31031D302C3C303D2C39
:10786000A831E520BC31031D372C78303D2C4B0E60
:10787000890C0339031D3E2CB430F107D710E41FE7
:10788000682C71082200EF0008309F310327BC31BB
:107890005A302200EF0007309F310327BC317108B6
:1078A00096316B26BC3197315E27BC31D7008731CA
:1078B0003827BC319F314027BC319531F525BC318B
:1078C0009F314D27BC3198317720BC318131D82987
:1078D000651C7D2C71082200EF000A309F310327C0
:1078E000BC315A302200EF0009309F310327BC31F0
:1078F00071089F31A427BC31632CE61FA22C7108AC
:107900002200EF000E309F310327BC315A30220095
:10791000EF000D309F310327BC31710896316B2683
:10792000BC3197314827BC31EF0087313827BC3153
:1079300097310B27BC319531F525BC319731302774
:10794000BC31662C671CBE2CFF30F1077108220089
:10795000EF0021004508803E9F310327BC31803075
:107960009531E325BC315A3A0319632C5A30220071
:10797000EF0080309F310327BC31632CE71C442D7E
:107980002A3071020318022D7108AF00FF30B001D8
:10799000AF07031CB003B2317C22BC312F08210099
:1079A000A300200030082100A4002000310821009D
:1079B000A50023082300E400210024082300E5009B
:1079C000210025082300E6009C31A824BC3164086E
:1079D0002200EF0014309F310327BC315A302200BF
:1079E000EF0013309F310327BC3187313827BC317A
:1079F0009631FE26BC319531F525BC3197312427CF
:107A0000BC31632C2A307102031C632C7108AF0057
:107A1000D630B001AF07031CB003B2317C22BC31B9
:107A20002F082100A000200030082100A100200024
:107A300031082100A20020082300E40021002108D1
:107A40002300E500210022082300E6009C31A82441
:107A5000BC3164082200EF0012309F310327BC3193
:107A60005A302200EF0011309F310327BC3187319B
:107A70003827BC319631F126BC319531F525BC3122
:107A800097311827BC31632CBB31172B2000D41F32
:107A90004E2D21000C110E102000D4133F305D0537
:107AA0002400CC003F3A031D6D2D2100C9012000A8
:107AB0006030D901DC01CB04A0309531E325BD3124
:107AC0005A3A031D692DA831EA20BD319F310327A1
:107AD000BD312000CA122100C80187317527BD3190
:107AE000CC36890B702D4C08031D962D0330740580
:107AF000CC00023A031D7F2D2000CC16812D2000E2
:107B0000CC12033074052400CC004C0B8A2D2000CD
:107B10004C168C2D20004C1274080339031D942D33
:107B20002100BB01BB0A962D2100BB012000CE1A0B
:107B30006E2EB731B627BD314F1C571D6E2EA030AB
:107B40009531E325BD315A3A031DAC2DA831EA2009
:107B5000BD319F310327BD31A2309531E325BD31C1
:107B6000003A0319B92D2200A230EF019F310327FB
:107B7000BD3187317527BD31CC36890BBC2D4C0802
:107B8000031D362E2000E819CB2D87315427BD3137
:107B9000031DD02DDC2D87315427BD31031DDC2D75
:107BA0007235A7313A27BD31AB0072082000D900E9
:107BB0002100D401D40AD50174082400CC0001307E
:107BC000CC36CC364C05CD002000680C2400CE000D
:107BD000CE0C4E0C01394D06CF0020004D0824007C
:107BE0004F06FE394F062000CD00CD1CF92D013087
:107BF000FA2D00302400CC0020004D1C012E013055
:107C0000022E003024004C0603190A2EA831A020B1
:107C1000BD314B1120004D1DCD1B172E87316F2715
:107C2000BD31CC364C082000DC004B19DC01720859
:107C3000A03E8600013087005C08A03E8400013031
:107C40008500000801020318272ECF15282ECF111A
:107C500087316F27BD31CC364C082100C800480859
:107C6000031D342E20004B118631892E8731752754
:107C7000BD31CC36890B392E4C038131031DF729D8
:107C8000BD312000D71C702EA831DC20BD31031D72
:107C9000702E210046087406031D702E2000BC3192
:107CA000C91B232C87316F27BD314C08F100200000
:107CB000501C5C2E4030F107D71071082100ED00F8
:107CC0009731D227BD319F310327BD317108220082
:107CD000EF0002309F3103278631842E8631982EA3
:107CE0008131EF290C122000501D892E21006E08D1
:107CF000F500590A7C2EF536890B7B2E7518822EDD
:107D000022000C162000E130501128009200910151
:107D1000080022000C1221005908031D0800200051
:107D2000D01021001312200013122800910192019B
:107D300020004E1BA22E8730D5055508F839023891
:107D4000D5000800A4260800CB2F2100C01C622FFC
:107D50002000550807390319622FEA27BE31093A76
:107D6000031DCA2E2100401CB82E21004015BA2E3A
:107D700021004011401DCA2E200055080739033A42
:107D80000319CE1EC52E4E17CA2E55080739013AC3
:107D90000319CE162000EA27BE310319DD2EEA278B
:107DA000BE31093A0319D62E6F27BE312000EA27CB
:107DB000BE31A900A903F027BE31EA27BE31031D59
:107DC000F72E55080739A900A90A55082906F839D8
:107DD0002906D50087394038D5000739033A031DF5
:107DE000F72EEA27BE31A900A90AF027BE31EA27FB
:107DF000BE31083A031D212F01309531E325BE31F4
:107E00005A3A031D082F02309531E325BE31092F60
:107E10003D302100ED00200055080739023A0319D2
:107E2000CE1E152F21003F081D2F55080739043A93
:107E300003194E1F212F21003D08CD00CD13B72778
:107E4000BE31200055080739053A031D622F210075
:107E50003F083D06031D362F3E083C06031D362F06
:107E6000E227BE31CF1350104E16602F3D093F065A
:107E7000031D422F3E083C06031D422FE227BE3160
:107E8000CF17332F3F083D06031D4F2FF927BE3173
:107E9000031D4F2FE227BE31CF135014342F3D095D
:107EA0003F06031D5B2FF927BE31031D5B2FE22721
:107EB000BE31CF174D2F2000CF1350104E12D710C8
:107EC000CA27BE312100C01C080020005508073910
:107ED000031D08005508F8390138D50008002100B5
:107EE00040187F2F8F2F2100BF0A8F2F2100BE0A3D
:107EF0008F2F2100BD0A8F2F2100BC0A8F2F200059
:107F000055080739013A0319732F033A0319762FDD
:107F1000013A0319792F073A03197C2F8F2F20007C
:107F2000550CA700A70C270C0F39A8000230280217
:107F3000031C0800A72F2100BF3508002100BE3513
:107F400008002100BD3508002100BC350800550897
:107F50000739013A03199B2F033A03199E2F013A5F
:107F60000319A12F073A0319A42FB62F08004D08B3
:107F70006D06031D08002000FB30D0142100EE0028
:107F800020001312280092019101210013160730DE
:107F9000D9000800CB2FF0302100C0052000D60109
:107FA000550887394838D500F830D5052100BF017C
:107FB000BE01BD01BC012000FF30CE124E132100D6
:107FC000EE0008003F082000DD0021003E08F4001C
:107FD00020000800550CA900A90C290C0F39080035
:107FE000A90DA90DA90D5508290687392906D5001F
:107FF0000800FC303C062000A90021003E060800D5
:020000040001F9
:08000E008C3FF635FF1FFF3F98
:08000000FF3FFF3FFF3FFF3F00
:10E00000D5005A003D00FF00FF00FF00FF00FF00A9
:10E01000FF00FF00FF00FF00FF00FF00FF00FF0008
:10E02000FF00FF00FF00FF00FF005A0003005A003E
:10E030000300FF00FF00FF00FF00FF00FF00FF00E4
:10E04000FF00FF00FF00FF00FF00FF00FF00FF00D8
:10E05000FF00FF00FF00FF00FF00FF00FF00FF00C8
:10E06000FF00FF00FF00FF00FF00FF00FF00FF00B8
:10E07000FF00FF00FF00FF005A0006005A000000EA
:10E08000FF00FF00FF00FF00FF00FF00FF00FF0098
:10E09000FF00FF00FF00FF00FF00FF00FF00FF0088
:10E0A000FF00FF005A000C00FF00FF00FF00FF0010
:10E0B000FF00FF00FF00FF00FF00FF00FF00FF0068
:10E0C000FF00FF00FF00FF00FF00FF00FF00FF0058
:10E0D000FF00FF00FF00FF00FF00FF00FF00FF0048
:10E0E000FF00FF00FF00FF00FF00FF00FF00FF0038
:10E0F000FF00FF00FF00FF00FF00FF00FF00FF0028
:10E10000FF00000000000000000000000000000010
:10E1100000000000000000000000000000000000FF
:10E1200000000000000000000000000000000000EF
:10E1300000000000000000000000000000000000DF
:10E14000FF00FF000000FF000000FF00FF000000D4
:10E15000FF000000FF00FF00FF00FF00FF00FF00C6
:10E16000FF00FF00FF00FF00FF00FF00FF00FF00B7
:10E17000FF00FF00FF00FF00FF00FF00FF00FF00A7
:10E18000FF00FF00FF00FF00FF00FF00FF00FF0097
:10E19000FF00FF00FF00FF00FF00FF00FF00FF0087
:10E1A000FF00FF00FF00FF00FF00FF00FF00FF0077
:10E1B000FF00FF00FF00FF00FF00FF00FF00FF0067
:10E1C000FF00FF00FF00FF00FF00FF00FF00FF0057
:10E1D000FF00FF00FF00FF00FF00FF00FF00FF0047
:10E1E000FF00FF00FF00FF00FF00FF00FF00FF0037
:10E1F000FF00FF00FF00FF00FF00FF00FF00FF0027
:00000001FF
